:020000040000FA
:06100000DAEF63F01200BC
:061008006EEF24F012005F
:06101800FCEF35F01200B0
:06102A00030021C80000D4
:1010300000050000E100000018C80000B70E000025
:101040000900000016C80000F307000002000000BD
:1010500002010000000000013200000000000180D9
:10106000004D0000000200000000000001320000FE
:1010700000000001A700FBFFDFFF015700EFFF04A6
:1010800000014E00F2FF0700014C00F3FF080001D1
:101090004A00F5FF0A00014400F8FF0B0001480078
:1010A000FAFF0D00014E00FCFF0F00015000FFFF92
:1010B000100001320000000A00012E0002000900A9
:1010C00001330002000A00012D0004000800012D78
:1010D0000004000800012F0005000800013100078E
:1010E000000700012E00070006000132000800067C
:1010F00000013300090005000136000A0004000168
:1011000034000A0003000139000B000300013D0018
:101110000C0002000141000D0001000146000E001C
:1011200001000146000E00FFFF0141000D00FFFF1E
:10113000013D000C00FEFF013E000C00FDFF0139E7
:10114000000B00FDFF0136000A00FCFF013300091F
:1011500000FBFF0132000800FAFF0135000800F92A
:10116000FF012E000600F9FF012E000600F9FF0125
:101170002D000400F8FF012D000400F8FF012E00EF
:101180000200F7FF012E000200F7FF01320000000D
:10119000F6FF012D000000F7FF012E00FEFFF7FF14
:1011A000012900FEFFF8FF012B00FDFFF8FF012FD2
:1011B00000FBFFF8FF012B00FBFFF9FF013100F9F5
:1011C000FFF9FF012E00F9FFFAFF013200F8FFFAE4
:1011D000FF013300F7FFFBFF013600F6FFFCFF01C4
:1011E0003900F5FFFDFF013900F5FFFDFF013D006E
:1011F000F4FFFEFF014100F3FFFFFF014600F2FF95
:10120000FFFF013200F6FF010001C60200008E0060
:10121000015B00EEFFFEFF015100F0FFFDFF014802
:1012200000F3FFFAFF014100F5FFF9FF013C00F771
:10123000FFF8FF013A00FAFFF6FF013600FCFFF667
:10124000FF013C00FFFFF4FF0128000100F8FF014F
:1012500029000200F8FF0126000300F9FF012B001E
:101260000500F9FF012E000700FAFF012F0008001A
:10127000FBFF0133000900FBFF013F000C00FCFFF6
:101280000100000000000002010000000000013227
:10129000000000000001CE003F006A0002000000D4
:1012A0000000000132000000000001120200009660
:1012B000FF0141000D000100013E000C0003000190
:1012C00034000A000300012F00080005000140005F
:1012D0000A000800013D0007000A00011B0002008F
:1012E0000500011B0002000500013C0001000C008C
:1012F000013700FFFF0B00012F00FDFF0900013641
:1013000000FAFF0900013500F9FF0800013D00F671
:10131000FF0700013C00F5FF0500014400F3FF0456
:1013200000014600F2FF0100010000000000000281
:1013300001000000000001320000000000019001E7
:1013400064FF4AFF020000000000000132000000BC
:10135000000001A200FBFFE0FF012D00F7FFFFFFEF
:10136000012600F9FFFDFF011D00FBFFFDFF01202D
:1013700000FBFFFCFF012700FBFFFAFF012B00FD34
:10138000FFF8FF012E00FEFFF7FF013200FFFFF61E
:10139000FF0132000100F6FF0133000200F6FF01F9
:1013A0002B000300F8FF0127000500FAFF012A00C7
:1013B0000600FAFF012B000700FBFF012B000800CD
:1013C000FDFF012F000900FDFF0160001300FEFF7B
:1013D000019B001F000000012B00F9FF0500012AFE
:1013E00000FAFF0600012700FBFF0600012800FCB1
:1013F000FF0700012400FCFF0600012400FEFF0798
:1014000000012800FFFF0800012800FFFF0800017D
:101410002D0001000900012D0001000900012F002D
:1014200003000900012D0004000800012800040049
:101430000700012E0006000700012E00070006002D
:1014400001320008000600013300090005000131E7
:1014500000090004000136000A0004000134000AFB
:10146000000300016B001500040001730017000168
:1014700000015000100000000151001000FEFF01AB
:1014800048000E00FDFF014A000E00FBFF014A006C
:101490000E00FBFF0141000B00F9FF0140000A00B4
:1014A000F8FF0139000800F8FF013D000700F6FFD2
:1014B000013C000500F5FF0138000200F5FF014185
:1014C000000100F3FF0128000000F8FF012900FEE1
:1014D000FFF8FF012400FEFFF9FF012800FCFFF9DF
:1014E000FF012800FCFFF9FF012E00FAFFF9FF01C0
:1014F0002E00F9FFFAFF012B00F9FFFBFF01870027
:101500001B0000000196000000E2FF01DE033AFF2D
:101510000000017D00E7FF0000016900EBFF020011
:10152000015600EFFF0300014400F3FF04000138FF
:1015300000F6FF0500013D00F6FF0700013500F849
:10154000FF0700013D00F9FF0A00013A00FAFF0A17
:1015500000013F00FCFF0C00013D00FEFF0C0001FC
:101560004600FFFF0E0001500001001000014E0078
:1015700004000F0001480006000D000144000800AF
:101580000B000120000400050001270006000500F3
:1015900001220006000300012600070003000124C9
:1015A0000007000200012900080002000155001197
:1015B0000001000100000000000002010000000026
:1015C000000132000000000001EA008A00E5FF028D
:1015D000000000000000013200000000000169006E
:1015E000EBFFFFFF015B00EEFFFDFF014F00F1FF8E
:1015F000FBFF012200FAFFFDFF012200FAFFFDFFC1
:10160000013C00F7FFF8FF013900F9FFF7FF013453
:1016100000FDFFF6FF013300FEFFF6FF0138000278
:1016200000F5FF0134000300F6FF0139000700F761
:10163000FF013C000900F8FF011D000500FDFF014E
:1016400026000700FDFF014A000E00FBFF015B00C2
:101650001200FDFF0164001400FFFF01640014008C
:10166000010001560011000300014F000F000500AA
:101670000145000C000700013C0009000800013989
:1016800000070009000131000400090001370001D2
:10169000000B00013200FFFF0A00013600FCFF0AC8
:1016A00000013900F9FF0900013C00F7FF080001C3
:1016B0004300F4FF0600014A00F2FF050001560056
:1016C000EFFF0300015F00EDFF01000100000000DB
:1016D00000000201000000000001320000000000D4
:1016E00001770176FF4EFF0200000000000001328A
:1016F000000000000001A200FBFFE0FF012D00F749
:10170000FFFFFF012600F9FFFDFF011D00FBFFFDAC
:10171000FF012000FBFFFCFF012700FBFFFAFF0198
:101720002B00FDFFF8FF012E00FEFFF7FF01320046
:10173000FFFFF6FF0132000100F6FF013300020057
:10174000F6FF012B000300F8FF0127000500FAFF58
:10175000012A000600FAFF012B000700FBFF012B06
:10176000000800FDFF012F000900FDFF01600013CC
:1017700000FEFF019B001F000000012B00F9FF0588
:1017800000012A00FAFF0600012700FBFF06000106
:101790002400FCFF0600012800FCFF0700012400D4
:1017A000FEFF0700012800FFFF0800012800FFFFDF
:1017B0000800012D0001000900012D0001000900B1
:1017C000012F000300090001280004000700012D7B
:1017D0000004000800012E0006000700012E00078B
:1017E0000006000132000800060001330009000570
:1017F00000013100090004000136000A0004000164
:1018000034000A000300016B00150004000173009E
:10181000170001000150001000FFFF0150001000F0
:10182000FFFF0148000E00FDFF014A000E00FBFF14
:10183000014A000E00FBFF0141000B00F9FF0140CF
:10184000000A00F8FF0139000800F8FF013D000719
:1018500000F6FF013C000500F5FF0138000200F52D
:10186000FF0141000100F3FF0128000000F8FF0123
:101870002900FEFFF8FF012400FEFFF9FF01280008
:10188000FCFFF9FF012800FCFFF9FF012E00FAFF21
:10189000F9FF012E00F9FFFAFF012B00F9FFFBFF12
:1018A0000187001B0000000196000000E2FF01DE3E
:1018B000033AFF0000017D00E7FF0000016900EB33
:1018C000FF0200015600EFFF0300014400F3FF0494
:1018D00000013800F6FF0500013D00F6FF0700019A
:1018E0003500F8FF0700013D00F9FF0A00013A004A
:1018F000FAFF0A00013F00FCFF0C00013D00FEFF63
:101900000C00014600FFFF0E000150000100100016
:10191000014E0004000F0001480006000D000144C4
:101920000008000B0001200004000500012400064F
:101930000004000124000600040001260007000343
:101940000001240007000200012900080002000134
:10195000550011000100010000000000000201001C
:10196000000000000132000000000001EA008A00CF
:10197000E5FF02000000000000013200000000004E
:10198000016900EBFFFFFF015B00EEFFFDFF014F70
:1019900000F1FFFBFF012200FAFFFDFF012200FA28
:1019A000FFFDFF013C00F7FFF8FF013900F9FFF7E9
:1019B000FF013400FDFFF6FF013800FEFFF5FF01D7
:1019C00033000200F6FF0134000300F6FF01390086
:1019D0000700F7FF013C000900F8FF011D000500AA
:1019E000FDFF0128000700FCFF0149000E00FCFF7D
:1019F000015B001200FDFF0164001400FFFF0164A1
:101A0000001400010001560011000300014F000FF7
:101A10000005000145000C000700013C000900081A
:101A2000000139000700090001310004000900012C
:101A3000370001000B00013200FFFF0A00013600F1
:101A4000FCFF0A00013900F9FF0900013C00F7FF23
:101A50000800014300F4FF0600014A00F2FF050000
:101A6000015600EFFF0300015F00EDFF01000100E0
:101A70000000000000020100000000000132000030
:101A8000000000018D0189FF32FF0200000000000C
:101A9000000132000000000001960000001E00015D
:101AA0002C063C01000001A5000000DFFF01300210
:101AB00090FF0000012B000700FBFF012A00060039
:101AC000FAFF0127000500FAFF0127000500FAFFD1
:101AD0000126000300F9FF0124000200F9FF0124A0
:101AE000000200F9FF0128000000F8FF012D0000AE
:101AF00000F7FF012900FEFFF8FF012900FEFFF8B3
:101B0000FF012D00FCFFF8FF012F00FBFFF8FF0194
:101B10002B00FBFFF9FF012E00F9FFFAFF012B005C
:101B2000F9FFFBFF012F00F8FFFBFF013100F7FF7A
:101B3000FCFF013600F6FFFCFF013400F6FFFDFF5D
:101B4000013900F5FFFDFF013C00F4FFFFFF0178C4
:101B500000E8FFFEFF014600F2FF0000014700F22F
:101B6000FF0200013D00F4FF0200013D00F4FF020E
:101B700000013B00F5FF0400013600F6FF04000100
:101B80003300F7FF0500013300F7FF0500013100C6
:101B9000F9FF0700012E00F9FF0600012B00FBFFF3
:101BA0000700012B00FBFF0700012D00FCFF0800D0
:101BB000012400FEFF0700012900FEFF0800012D9F
:101BC00000000009000128000000080001290002AF
:101BD000000800012600030007000126000300079B
:101BE0000001270005000600012A0006000600018A
:101BF0002E0007000600012F0008000500019100DB
:101C0000E3FF0000020100000000000132000000BC
:101C1000000001C10074000000020000000000008C
:101C200001320000000000015F00EDFFFFFF0150E6
:101C300000F0FFFFFF014800F2FFFDFF013600F654
:101C4000FFFCFF012800F9FFFCFF012700FAFFFB62
:101C5000FF012000FBFFFCFF012300FBFFFBFF0156
:101C60002200FDFFFAFF011B00FEFFFBFF01200029
:101C7000FEFFFAFF0123000000F9FF01320001001E
:101C8000F6FF0131000400F7FF0139000700F7FFFC
:101C90000140000A00F8FF0145000C00F9FF015463
:101CA000001000FBFF0156001100FDFF0169001547
:101CB00000FFFF01690015000100015B0012000335
:101CC00000014F000F000500012200060003000183
:101CD000220006000300013C000900080001350055
:101CE0000700080001360004000A0001320001006C
:101CF0000A00013200FFFF0A00013600FCFF0A0063
:101D0000013900F9FF0900014000F6FF0800014316
:101D100000F4FF0600014F00F1FF0500015600EF3F
:101D2000FF0300016400ECFF01000100000000005F
:101D3000000201000000000001320000000000016C
:101D40001001FFFF5DFF02000000000000013200F3
:101D500000000000014B000F00FFFF0146000E00D5
:101D6000FFFF0148000E00FDFF013E000C00FDFFDB
:101D7000013B000B00FCFF013C000B00FBFF0136A8
:101D8000000900FAFF0135000800F9FF012A0006EA
:101D900000FAFF012B000500F9FF0128000400F9FB
:101DA000FF0128000400F9FF012B000300F8FF01E8
:101DB00029000200F8FF0128000100F8FF012D00B2
:101DC0000000F7FF0132000000F6FF012E00FEFFC9
:101DD000F7FF012E00FEFFF7FF012B00FDFFF8FFCC
:101DE000012F00FBFFF8FF012B00FBFFF9FF012E85
:101DF00000FAFFF9FF013200F8FFFAFF013200F8A4
:101E0000FFFAFF012F00F8FFFBFF013800F6FFFB90
:101E1000FF013400F6FFFDFF013900F5FFFDFF0172
:101E20003D00F4FFFEFF014100F3FFFFFF01410011
:101E3000F3FF0000016900EBFF0000016000EDFF0F
:101E40000200015200F0FF0400014A00F2FF050009
:101E5000014300F4FF0600013D00F6FF07000140CA
:101E600000F7FF0900014000F8FF0A00013F00FAF7
:101E7000FF0B00013C00FBFF0B00013D00FEFF0CCF
:101E800000013C00FFFF0C0001320000000A0001CD
:101E90002E0002000900012E0002000900012D00A1
:101EA00004000800012D0004000800012F000500B7
:101EB0000800012E0007000600013100070007009E
:101EC0000132000800060001330009000500013658
:101ED000000A0004000134000A000300013E000C67
:101EE000000300013D000C0002000146000E00014D
:101EF000000146000E000100010000000000000289
:101F00000100000000000132000000000001390063
:101F10000000DEFF020000000000000132000000AF
:101F20000000016900EBFFFFFF015B00EEFFFDFF1A
:101F3000014F00F1FFFBFF012200FAFFFDFF01242A
:101F400000FAFFFCFF014000F6FFF8FF013D00F939
:101F5000FFF6FF013600FCFFF6FF013C00FFFFF437
:101F6000FF013C000100F4FF0136000400F6FF0110
:101F70003D000700F6FF0140000A00F8FF012400C1
:101F80000600FCFF0122000600FDFF0154001000C6
:101F9000FBFF015B001200FDFF0169001500FFFF60
:101FA0000164001400010001560011000300014FFC
:101FB000000F0005000126000700030001200005B6
:101FC0000004000143000A0009000139000700096C
:101FD00000013B0004000B0001370001000B000171
:101FE0003C00FFFF0C00013600FCFF0A00013D0031
:101FF000F9FF0A00014000F6FF0800012000FBFF86
:102000000400012600F9FF0300014F00F1FF050065
:10201000015B00EEFF0300016400ECFF0100010022
:10202000000000000002010000000000013200007A
:1020300000000001BC01B0FF02FF02000000000030
:10204000000132000000000001AC00DEFFFBFF01D8
:102050004300FDFF0D00013C00FFFF0C00012800C4
:102060000100080001230001000700012400020014
:102070000700011D00030005000119000300040012
:102080000120000500040001190004000300011DE7
:102090000005000300012300070001000133000ACE
:1020A0000002000191001D00010001940284000063
:1020B00000017300000017000196001E00000001DF
:1020C00073000000E9FF011D013900000001C90093
:1020D0001700DFFF019001B0FF000001A000000029
:1020E000E0FF019600E2FF000001A00000002000D8
:1020F000019E027AFF0000014600F2FF000001236A
:1021000000F9FFFFFF011D00FBFFFDFF011500FDB2
:10211000FFFDFF011B00FEFFFBFF011E00FFFFFA9A
:10212000FF0147000200F2FF010000000000000272
:10213000010000000000013200000000000158070B
:102140005AFF5C04020000000000000132000000A1
:10215000000001C701A8FFE9FF0141000000F3FFF3
:10216000015C014400F1FF014C00F1FFFEFF011092
:1021700001CBFFF4FF0141000000F3FF01C701584C
:1021800000E9FF013C0000000C00010701CDFF0D3C
:1021900000015700EFFF0400015700110004000187
:1021A000050133000B00013C0000000C000106019A
:1021B000CDFF0C00016100EDFF0400016100130080
:1021C000040001060133000C0001410000000D0075
:1021D00001000000000000020100000000000132C8
:1021E000000000000001FF00A8FF83FF02000000C4
:1021F0000000000132000000000001C60158001676
:10220000000141000000F3FF010501CDFFF5FF01D2
:102210006200EDFFFBFF0161001300FCFF010501FF
:102220003300F5FF0141000000F3FF010501CDFF80
:10223000F5FF015700EFFFFCFF0157001100FCFF05
:102240000107013300F3FF013C000000F4FF01C768
:1022500001A8FF170001410000000D000110013529
:10226000000C00014C000F000300015C01BCFF0FDB
:102270000001410000000D0002010000000000010B
:1022800032000000000001AC00000099FF020000D5
:10229000000000000132000000000001C6015800EB
:1022A0001600013C000000F4FF010601CDFFF4FF21
:1022B000016200EDFFFBFF0160001300FDFF01065E
:1022C000013300F4FF0141000000F3FF010501CDDF
:1022D000FFF5FF015700EFFFFCFF0157001100FC65
:1022E000FF0107013300F3FF013C000000F4FF0190
:1022F000C701A8FF170001410000000D00011001F7
:1023000035000C00014C000F000300015C01BCFF14
:102310000F0001410000000D00020100000000005C
:1023200001320000000000019B000000A3FF02003A
:102330000000000000013200000000000155001103
:102340000000000146000000F2FF015500EFFF0011
:102350000001460000000E00020100000000000124
:102360003200000000000197001C00AAFF020000DC
:102370000000000001320000000000014100FFFFEA
:10238000F3FF012400F9FF0200012000FAFF020020
:10239000011900FCFF0300012000FBFF0400011DE8
:1023A00000FDFF0500011B00FEFF0500011B00FEF4
:1023B000FF0500011E0000000600012800010008C2
:1023C00000012400020007000124000400060001AF
:1023D00023000500050001240006000400012B0075
:1023E00008000300012E00090002000132000A006B
:1023F00000000137000B000000012E000900FEFF65
:10240000012B000800FDFF0128000700FCFF01234D
:10241000000500FBFF0124000400FAFF0126000371
:1024200000F9FF0123000000F9FF0123000000F97B
:10243000FF012200FDFFFAFF012200FDFFFAFF016C
:102440002700FAFFFBFF012400FAFFFCFF012B002D
:10245000F8FFFDFF012E00F7FFFEFF013700F5FF3B
:10246000FFFF011500FCFF01000113010000370010
:10247000012300F9FFFFFF012000FAFFFEFF011B0F
:1024800000FBFFFEFF011600FCFFFEFF011900FD2F
:10249000FFFCFF011500FDFFFDFF011500FFFFFC24
:1024A000FF011900FFFFFBFF011E000100FAFF0101
:1024B00020000400FBFF0123000500FBFF012B00AF
:1024C0000800FDFF01000000000000020100000004
:1024D0000000013200000000000150001900290036
:1024E000020000000000000132000000000001CDE9
:1024F000000000D7FF012D000900010001260007A0
:10250000000300011C000400040001150003000387
:10251000000116000200040001190000000500017E
:10252000140000000400011600FEFF040001120068
:10253000FEFF0300011500FDFF0300011900FCFF71
:102540000300011600FCFF0200011900FBFF01005F
:10255000011900FBFF010001000000000000020162
:10256000000000000001320000000000019700C4DC
:10257000FFBCFF020000000000000132000000006C
:1025800000013E00FDFFF4FF011900FBFFFFFF010A
:102590001900FCFFFDFF011D00FDFFFBFF012900ED
:1025A000FEFFF8FF0124000200F9FF0122000300F2
:1025B000FAFF0120000500FCFF0120000600FEFFDD
:1025C0000123000700FFFF0141000D00000001246E
:1025D00000FAFF0400011D00FDFF0500011B00FEC5
:1025E000FF0500011E00FFFF060001230001000798
:1025F0000001240002000700012000040005000182
:1026000027000600050001260007000300012B003B
:102610000800030001280008000100012D00090046
:102620000100013C000C00FFFF0139000B00FDFF21
:102630000138000A00FBFF012E000700FAFF011617
:10264000000200FCFF0116000200FCFF0115000162
:1026500000FCFF0119000000FBFF011E000000FA52
:10266000FF012200FDFFFAFF012000FCFFFBFF013C
:102670002300FBFFFBFF0132000A000000013700CE
:102680000000F5FF017C01B4FF0000015A00EEFFDD
:102690000100011E00FAFF0100011900FBFF01000B
:1026A000012F00F8FF0500012E00FAFF0700012DA1
:1026B00000FCFF0800013200FFFF0A0001230001B7
:1026C00000070001190001000500011B00020005C0
:1026D00000011D00030005000119000400030001B2
:1026E0001D0005000300011E00060001000123007B
:1026F00007000000010000000000000201000000CF
:10270000000001320000000000015A003500F6FF11
:10271000020000000000000132000000000001285B
:1027200000F8FF0000012300F9FFFFFF012000FA7D
:10273000FFFEFF011D00FBFFFDFF011500FDFFFD7A
:10274000FF011500FDFFFDFF011500FFFFFCFF016C
:102750001500FFFFFCFF0115000100FCFF01150043
:102760000100FCFF0115000300FDFF01190003003B
:10277000FCFF011B000500FEFF0120000600FEFF1C
:10278000011E000600FFFF012800080000000128CC
:102790000008000000011E000600010001200006E4
:1027A000000200011D0005000300011500030003E5
:1027B00000011500030003000115000100040001E1
:1027C000150001000400011500FFFF0400011500C1
:1027D000FFFF0400011500FDFF0300011500FDFFD0
:1027E0000300011D00FBFF0300011B00FBFF0200B3
:1027F000012300F9FF0100012300F9FF000001009F
:102800000000000000020100000000000132000092
:10281000000000019100CBFFBBFF020000000000A0
:102820000001320000000000013E00FDFFF4FF0146
:102830001900FBFFFFFF011900FCFFFDFF01220053
:10284000FDFFFAFF012400FEFFF9FF01290002004D
:10285000F8FF011D000300FBFF0120000500FCFF45
:102860000122000600FDFF012300070000000141D6
:10287000000D00FFFF012700FAFF0500011D00FD0C
:10288000FF0500011B00FEFF0500011E00FFFF0603
:1028900000012300010007000120000200060001E2
:1028A00024000400060001240006000400012800A2
:1028B00007000400012B00080003000128000800A5
:1028C0000100012D0009000100013C000C00FFFF88
:1028D0000139000B00FDFF0138000A00FBFF012E4B
:1028E000000700FAFF0116000200FCFF01160002BB
:1028F00000FCFF0115000100FCFF0119000000FBB6
:10290000FF011E000000FAFF012200FDFFFAFF0197
:102910002000FCFFFBFF012300FBFFFBFF01320057
:102920000A0000000137000000F5FF017C01B4FF40
:102930000000015A00EEFF0100011E00FAFF010035
:10294000011900FBFF0100012F00F8FF0500012A1B
:1029500000FAFF0600013100FCFF0900013200FF10
:10296000FF0A00011E0001000600011E0001000612
:1029700000011B0002000500011900030004000112
:102980001C0004000400011B0005000200012000DF
:102990000600020001230007000000010000000003
:1029A00000000201000000000001320000000000F1
:1029B000015A003500F6FF0200000000000001325D
:1029C0000000000000012800F8FF0000012400F9C9
:1029D000FFFEFF011E00FAFFFFFF011D00FBFFFDD0
:1029E000FF011500FDFFFDFF011500FDFFFDFF01CB
:1029F0001500FFFFFCFF011500FFFFFCFF011500A4
:102A00000100FCFF0115000100FCFF01190003009B
:102A1000FCFF0115000300FDFF011B000500FEFF88
:102A20000120000600FEFF011E000600FFFF012836
:102A3000000800FFFF01280008000100011E000639
:102A400000010001200006000200011B0005000239
:102A50000001190003000400011500030003000138
:102A6000150001000400011500010004000115001B
:102A7000FFFF0400011500FFFF0400011500FDFF2A
:102A80000300011500FDFF0300011D00FBFF030013
:102A9000011900FBFF0100012400F9FF02000123DE
:102AA00000F9FF000001000000000000020100002A
:102AB00000000001320000000000016F00F7FFBEBF
:102AC000FF020000000000000132000000000001D1
:102AD0004B000F00000001C3000000D9FF014B00B4
:102AE000F1FF000001C30000002700020100000008
:102AF000000001320000000000017B00DBFFC0FF8E
:102B00000200000000000001320000000000013758
:102B10000000000B000162027A000000013C00008E
:102B200000F4FF01DC00D4FF00000124000600FCDB
:102B3000FF011D000300FBFF011D000300FBFF015F
:102B40001E000000FAFF0123000000F9FF0122002F
:102B5000FDFFFAFF012400FCFFFAFF012000FBFF4C
:102B6000FCFF012800F9FFFCFF012900F8FFFEFF30
:102B7000012900F8FFFEFF012D00F7FFFFFF0137DD
:102B800000F5FF0100013300F6FF0200012B00F801
:102B9000FF0300012800F9FF0400012300FBFF05EB
:102BA00000012000FCFF0500012000FEFF060001DF
:102BB0001E00FFFF0600011E0001000600012000AC
:102BC00002000600012000040005000124000600A8
:102BD0000400013700F5FF000002010000000000C2
:102BE00001320000000000014B002D000000020037
:102BF000000000000001320000000000014600F269
:102C0000FFFFFF012F00F7FFFDFF011D00FBFFFD90
:102C1000FF011C00FCFFFCFF011600FEFFFCFF0192
:102C20001900FFFFFBFF0115000100FCFF01100070
:102C30000100FDFF0119000300FCFF011900040061
:102C4000FDFF011B000500FEFF011B000500FEFF4C
:102C50000123000700FFFF0128000800FFFF0128F3
:102C6000000800010001230007000100011E00060A
:102C7000000100011D000500030001150003000311
:102C8000000115000300030001160002000400010A
:102C900014000000040001140000000400011200F0
:102CA000FEFF0300011900FDFF0400011500FDFFF8
:102CB0000300011D00FBFF0300011E00FAFF0100DD
:102CC000012400F9FF0200012300F9FF00000100C8
:102CD00000000000000201000000000001320000BE
:102CE000000000016900FFFFC1FF020000000000BA
:102CF0000001320000000000013C000C00FFFF0159
:102D000033000A00FEFF012D000800FCFF012B002C
:102D10000700FBFF0120000400FBFF011D00030072
:102D2000FBFF0120000200FAFF0123000000F9FF71
:102D30000123000000F9FF012600FDFFF9FF011D3E
:102D400000FDFFFBFF012A00FAFFFAFF012400FA51
:102D5000FFFCFF012B00F8FFFDFF012E00F7FFFE37
:102D6000FF013200F6FF0000014B00F1FF010001FE
:102D70001E00FAFF0100011B00FBFF0200013300EF
:102D8000F7FF0500013100F9FF0700013100FCFFEA
:102D90000900012D00FFFF090001280001000800C3
:102DA00001200002000600012400040006000123A7
:102DB000000500050001240006000400012B0008A6
:102DC0000003000133000A0002000132000A000182
:102DD00000010000000000000201000000000001EE
:102DE0003200000000000116000000F3FF020000A6
:102DF0000000000001320000000000012800F8FF80
:102E00000000012400F9FFFEFF011E00FAFFFFFF92
:102E1000011900FCFFFDFF011900FCFFFDFF011976
:102E200000FDFFFCFF011500FFFFFCFF011900FF83
:102E3000FFFBFF0115000100FCFF0115000100FC74
:102E4000FF0119000300FCFF0119000400FDFF0150
:102E50001D000500FDFF011B000500FEFF0128000D
:102E60000800FFFF01280008000000012300070000
:102E700000000123000700010001200006000200FD
:102E8000011D0005000300011500030003000119E6
:102E900000030004000115000100040001150001F9
:102EA000000400011900FFFF0500011500FFFF04E9
:102EB00000011900FDFF0400011500FDFF030001E2
:102EC0001D00FBFF0300011E00FAFF0100012400AA
:102ED000F9FF0200012800F8FF00000100000000D7
:102EE00000000201000000000001320000000000AC
:102EF00001AB00E1FF9EFF02000000000000013274
:102F00000000000000014200F3FFFEFF012D00FF62
:102F1000FF0900011E0000000600011B0002000561
:102F20000001150003000300011600040002000167
:102F30002300070001000137000B00010001FF0022
:102F400033000000012D00000009000137000B00D4
:102F50000000012D000000F7FF016E0016000000C8
:102F6000014F000900F3FF019B00E1FF0000013C5D
:102F7000000000F4FF013700F5FF0000013C0000F5
:102F8000000C00010401CCFF0000012800F8FF0044
:102F900000011500FDFFFDFF011500FFFFFCFF0113
:102FA00019000000FBFF010000000000000201000A
:102FB0000000000001320000000000012200F3FFC9
:102FC000F0FF0200000000000001320000000000DD
:102FD000015500110000000146000000F2FF0155FC
:102FE00000EFFF000001460000000E00020100009B
:102FF000000000013200000000000196002000AC3B
:10300000FF0200000000000001320000000000018B
:103010003D00FEFFF4FF012300F9FF010001200045
:10302000FAFF0200012200FAFF0300011C00FCFF6E
:103030000400011C00FCFF0400011D00FDFF050051
:10304000012000FEFF060001190000000500012814
:103050000001000800012000020006000124000415
:1030600000060001230005000500012400060004FD
:1030700000012B0008000300012D000900010001E0
:1030800037000B0001000141000D00FFFF013E0071
:103090000C00FDFF011B000500FEFF0119000400EC
:1030A000FDFF0119000400FDFF0119000300FCFFF2
:1030B000012D000400F8FF0132000100F6FF0119A4
:1030C000000000FBFF011E00FFFFFAFF011900FDD9
:1030D000FFFCFF011900FDFFFCFF011C00FCFFFCD1
:1030E000FF011D00FBFFFDFF011B00FBFFFEFF01B9
:1030F0002300F9FFFFFF013D00FEFF0C0001290046
:103100000800020001240006000400011D00030065
:103110000500011E0001000600011400000004006B
:10312000011600FEFF0400011900FDFF0400011557
:1031300000FDFF0300011D00FBFF0300012000FA5A
:10314000FF0200012300F9FF0100012800F8FF0041
:1031500000012800F8FF0000012300F9FFFFFF0134
:103160002000FAFFFEFF011D00FBFFFDFF0115001F
:10317000FDFFFDFF011500FDFFFDFF011500FFFF35
:10318000FCFF011500FFFFFCFF0124000200F9FF16
:103190000124000400FAFF0112000300FEFF0116E3
:1031A000000400FEFF012E000900FEFF01000000E8
:1031B00000000002010000000000013200000000D9
:1031C000000124000C00EEFF0200000000000001DE
:1031D000320000000000013C000C00FFFF01330042
:1031E0000A00FEFF012D000800FCFF012B00070074
:1031F000FBFF0120000400FBFF011D000300FBFF9B
:103200000120000200FAFF0123000000F9FF012362
:10321000000000F9FF012600FDFFF9FF012200FD7B
:10322000FFFAFF012700FAFFFBFF012400FAFFFC71
:10323000FF012B00F8FFFDFF012E00F7FFFEFF014D
:103240003200F6FF0000014B00F1FF0100011E00FB
:10325000FAFF0100011B00FBFF0200013300F7FF32
:103260000500013100F9FF0700013100FCFF0900F2
:10327000012D00FFFF0900012300010007000124C8
:1032800000020007000124000400060001230005DD
:1032900000050001240006000400012B00080003C3
:1032A000000133000A0002000132000A000100019F
:1032B00000000000000002010000000000013200D8
:1032C000000000000116000000F3FF0200000000F3
:1032D000000001320000000000012800F8FFFFFF9D
:1032E000012300F9FFFFFF012000FAFFFEFF011696
:1032F00000FCFFFEFF011C00FCFFFCFF011500FDB0
:10330000FFFDFF011500FFFFFCFF011900FFFFFBA0
:10331000FF0115000100FCFF0115000100FCFF0189
:1033200019000300FCFF0119000400FDFF011D004E
:103330000500FDFF011B000500FEFF01280008003D
:10334000FFFF0128000800FFFF0123000700010024
:103350000123000700010001200006000200011DFA
:10336000000500030001150003000300011900031C
:103370000004000115000100040001150001000413
:1033800000011900FFFF0500011500FFFF04000107
:103390001500FDFF0300011900FDFF0400011B00E3
:1033A000FBFF0200012000FAFF0200012300F9FFE9
:1033B0000100012800F8FF010001000000000000EA
:1033C0000201000000000001320000000000018B3B
:1033D00000D4FFB9FF02000000000000013200002D
:1033E00000000001B801580000000137000000F59E
:1033F000FF013C00F4FF00000124000600FCFF0177
:1034000024000400FAFF0122000300FAFF01230058
:103410000100F9FF012300FFFFF9FF012200FDFF7A
:10342000FAFF012300FBFFFBFF012000FAFFFEFF74
:10343000012B000700FBFF0127000500FAFF012018
:10344000000200FAFF011E000100FAFF011900004E
:1034500000FBFF011900FFFFFBFF011900FDFFFC4E
:10346000FF011500FDFFFDFF011900FCFFFDFF013D
:103470001B00FBFFFEFF011E00FAFFFFFF01230000
:10348000F9FF0000013101C3FF0000013C00000012
:103490000C000118013800000001230007000100A2
:1034A000011E0006000100011000030001000115CB
:1034B00000030003000116000200040001140000D4
:1034C000000400010F0000000300011500FFFF04CD
:1034D00000011200FEFF0300011200FDFF020001C7
:1034E0001500FDFF0300011900FBFF0100013D0075
:1034F000F4FF020001FF00CDFF0000013C000000CE
:103500000C00011D0139000000012D00090001001F
:103510000120000600020001120003000200010B5E
:103520000001000200011E00010006000119000058
:10353000000500011D00FDFF0500011C00FCFF044B
:1035400000012000FAFF0200012900F8FF0200013B
:103550003200F6FF000001E600D2FF00000141004A
:1035600000000D0002010000000000013200000018
:10357000000001ED05CB0089FC0200000000000006
:103580000132000000000001A400F5FFE1FF01A1ED
:1035900000F7FFE1FF012201F1FFC8FF010501F57E
:1035A000FFCDFF01DA00F9FFD5FF01B100FBFFDD20
:1035B000FF018700FEFFE5FF016E00FEFFEAFF024C
:1035C0000100000000000132000000000001F801CD
:1035D0003E0028010200000000000001320000004F
:1035E000000001800280FF000002010000000000D6
:1035F00001320000000000010C02EC0030FF02006C
:1036000000000000000132000000000001AB00F7E4
:10361000FF2100019500F6FF1C00019600F5FF1C3C
:1036200000019D00F4FF1D0001C000F0FF23000118
:10363000CE00ECFF2400016300F6FF1100016100E1
:10364000F5FF1000016400F4FF1000016000F4FFBA
:103650000F00012A00FAFF0600012700FAFF05000B
:10366000012400FAFF0400012000FAFF02000120FB
:1036700000FAFF0200011E00FAFF0000013C00F406
:10368000FF0000013D00F4FFFEFF014200F3FFFEDA
:10369000FF014200F3FFFEFF014600F2FF000001C0
:1036A0003700F5FF0000012D00F7FFFFFF012B00A1
:1036B000F8FFFDFF012000FBFFFCFF010E00FEFFF5
:1036C000FEFF010F000000FDFF011000FFFFFDFFE6
:1036D0000115000100FCFF012D000400F8FF01406E
:1036E000000800F6FF0120000400FBFF0124000297
:1036F00000F9FF012E000200F7FF012D000000F786
:10370000FF012D00FFFFF7FF012E00FEFFF7FF0175
:103710002800FCFFF9FF012700FBFFFAFF02010070
:103720000000000001320000000000019E02FF00C6
:10373000C9FE02000000000000013200000000008D
:10374000011E000600000001150004000100011226
:10375000000300020001160002000400011B000229
:1037600000050001190001000500014600FFFF0EE1
:1037700000014C00FEFF0F00014C00FDFF0F000197
:103780008E00FBFF1C00018F00FAFF1C00020100ED
:103790000000000001320000000000012902E9FEE3
:1037A000B400020000000000000132000000000030
:1037B000015D00EEFFFBFF014700F2FFFEFF013756
:1037C00000F5FF0000012F00F7FF0300012700FABA
:1037D000FF0500012700FBFF0600012600FDFF0793
:1037E00000012E00FEFF0900015600FDFF1100013F
:1037F0002D00FFFF0900012900FEFF08000126003F
:10380000FDFF0700012000FCFF0500012400FAFF76
:103810000400012800F8FF0100018A01EFFFB3FF57
:10382000011E000000FAFF0119000100FBFF013634
:10383000000400F6FF013A000600F6FF013600061C
:1038400000F7FF0160000C00F1FF0128000400F9FF
:10385000FF0120000200FAFF010B00FFFFFEFF0145
:103860001000FFFFFDFF012E00F9FFFAFF018A00A3
:10387000EBFFEEFF014B00F4FFF7FF014A00F6FFFC
:10388000F5FF014300F7FFF6FF011D00FDFFFBFF01
:10389000011B00FEFFFBFF014B01F3FFBFFF010413
:1038A00001F6FFCDFF011900050000000119000518
:1038B00000010001160004000200011600040002CD
:1038C0000001350007000800013A0006000A000167
:1038D00094000C001B00015E000800110001600054
:1038E00009001100011D0003000500011C00040077
:1038F00004000144000B000800014A000D0007000D
:10390000014A000E0005000147000E0002000123DD
:1039100000070000000123000700FFFF0120000650
:1039200000FEFF011D000500FDFF0120000500FC59
:10393000FF0124000400FAFF0131000400F7FF0139
:103940003E000300F4FF0141000100F3FF014600C7
:103950000000F2FF02010000000000013200000040
:103960000000010A00060000000200000000000044
:103970000132000000000001660014000400015143
:103980000010000200013C000C0000000133000A9E
:1039900000FEFF012D000800FCFF0132000800FAC4
:1039A000FF0135000800F9FF0143000900F6FF019F
:1039B0004E000A00F4FF014E000A00F4FF019E00D1
:1039C0001200E6FF0138012100CBFF01550008007D
:1039D000F1FF015C000900F0FF01BE000F00DDFFF8
:1039E00001BF000D00DCFF01B1000A00DEFF01F79E
:1039F000000C00D0FF01F5000A00D0FF015A0001C1
:103A000000EEFF011E00FFFFFAFF011500FFFFFCA3
:103A1000FF011200FEFFFDFF011200FDFFFEFF018E
:103A20001000FDFFFFFF011000FDFF0100012E004F
:103A3000F7FF0200012F00F7FF0300013900F5FF37
:103A40000300013200F6FF0100013200F6FF000022
:103A5000012E00F7FF0200013100F7FF04000136DC
:103A600000F7FF0600013900F7FF0700013C00F8EE
:103A7000FF0900014300F7FF0A00014400F8FF0BB3
:103A800000018900F1FF1700019200F1FF19000108
:103A90008B00F2FF1800018000F3FF160002010006
:103AA0000000000001320000000000019B01C4FF83
:103AB000EF000200000000000001320000000000E2
:103AC000015F00EDFF0000015100F0FFFEFF013D2E
:103AD00000F4FFFEFF013100F7FFFCFF011500FDC0
:103AE000FFFDFF011500FDFFFDFF011600FEFFFCBD
:103AF000FF011500FFFFFCFF013C00FFFFF4FF0189
:103B00004C000200F1FF0156000300EFFF016100CD
:103B10000400EDFF0162000500EDFF0165000700F4
:103B2000EDFF0165000900EEFF0132000600F8FF1D
:103B30000132000600F8FF0135000700F8FF0131EF
:103B4000000700F9FF0132000800FAFF0133000905
:103B500000FBFF0201000000000001320000000035
:103B600000011D00F1FF090002000000000000013B
:103B700032000000000001FF00F6FFCEFF015601F9
:103B8000F2FFBDFF02010000000000013200000052
:103B900000000186023D01DF00020000000000007D
:103BA00001320000000000019300F7FFE4FF0182F2
:103BB00000F9FFE7FF010701F3FFCDFF019F00F9C7
:103BC000FFE1FF01C500FAFFD9FF01D400FAFFD6DB
:103BD000FF01DD00FCFFD4FF020100000000000136
:103BE000320000000000018F01F7FFEF000200002B
:103BF0000000000001320000000000017F000B0007
:103C0000E9FF014600F2FFFFFF017D00F6FF17000C
:103C10000141000D00010001000000000000020150
:103C2000000000000001320000000000011700F257
:103C3000FF00000200000000000001320000000050
:103C400000016A00FDFFEBFF0172000900EBFF01BC
:103C50005D000500120002010000000000013200BA
:103C600000000000012700F4FF1400020000000023
:103C7000000001320000000000014F01BDFFFFFF06
:103C80000201000000000001320000000000016E8F
:103C9000004000EFFF0200000000000001320000C1
:103CA000000000010901CBFF00000201000000003C
:103CB0000001320000000000016F003F00EBFF0236
:103CC0000000000000000132000000000001FA00C6
:103CD000CEFF0000020100000000000132000000E1
:103CE00000000179003A002C0002000000000000F2
:103CF0000132000000000001F2021D0094000201E8
:103D0000000000000001320000000000010401D5A5
:103D1000FF6AFF0200000000000001320000000006
:103D20000001F7021D0095000201000000000001E3
:103D3000320000000000011D01FCFF55FF020000E1
:103D4000000000000132000000000001BF021B0063
:103D50008A000201000000000001320000000000A3
:103D6000012B0002001A00020000000000000132D6
:103D70000000000000012800FFFF0800012400FEF1
:103D8000FF0700010700FFFF0100010700FFFF011F
:103D900000010E00FEFFFEFF012800FCFFF9FF02FC
:103DA00001000000000001320000000000011800C6
:103DB000F2FFFEFF020000000000000132000000E0
:103DC00000000124000200070001150003000300A9
:103DD000010B00020001000141000D000000020182
:103DE00000000000000132000000000001EF007A36
:103DF000FF3300020000000000000132000000005C
:103E0000000126000700FDFF0126000700FDFF015D
:103E100032000800FAFF012E000700FAFF0135000A
:103E20000700F8FF0136000600F7FF013600060024
:103E3000F7FF013A000600F6FF0138000500F6FF23
:103E4000013B000400F5FF0139000300F5FF0133D9
:103E5000000200F6FF0137000100F5FF012D000010
:103E600000F7FF013200FFFFF6FF012D00FCFFF815
:103E7000FF012600FDFFF9FF012300FBFFFBFF010F
:103E80001D00FBFFFDFF012200FAFFFDFF011E00E8
:103E9000FAFFFFFF011E00FAFFFFFF011E00FAFFFD
:103EA0000100012300F9FF0100013F00F4FF0400BD
:103EB000014300F4FF0600013900F7FF0700013558
:103EC00000F8FF07000201000000000001320000BE
:103ED00000000001F30085003C000200000000002B
:103EE000000132000000000001D600D7FFF4FF02FD
:103EF000010000000000013200000000000140004D
:103F00002500F5FF02000000000000013200000063
:103F1000000001C100DBFF0B0002010000000000F7
:103F200001320000000000016B003F000C000200A5
:103F300000000000000132000000000001400140CC
:103F40000000000136013E0000000176027E00FD07
:103F5000FF014C000F00FEFF012D000900FFFF01D3
:103F600010000300FFFF010B000100FEFF01100025
:103F70000100FDFF0119000000FBFF012800FFFF09
:103F8000F8FF010B00FFFFFEFF010B00FEFFFFFF2C
:103F9000012D00F7FFFFFF015000F0FFFFFF017B45
:103FA0000281FF0100013B01C1FF0100014001C08E
:103FB000FF0300010B00FEFF0100010E00FEFF02E7
:103FC00000011500FFFF04000119000000050001B9
:103FD0001900010005000115000100040001120094
:103FE00002000300011000030001000100000000B6
:103FF000000002010000000000013200000000008B
:104000000147001500DBFF02000000000000013244
:10401000000000000001BA00EFFFDFFF015900F8C7
:10402000FFF0FF015E00F8FFEFFF0201000000005B
:104030000001320000000000016D00EBFFC2FF0232
:1040400000000000000001320000000000016200DA
:10405000FBFFEDFF016000FEFFEDFF016000FEFFD2
:10406000EDFF015F00FFFFEDFF01C3000100D9FF7D
:1040700001B9000100DBFF02010000000000013275
:104080000000000000015B014300C50002000000C9
:104090000000000132000000000001C800D8FFFF4E
:1040A000FF020100000000000132000000000001DA
:1040B0005002EBFE22FF020000000000000132006F
:1040C0000000000001280008000100012600070090
:1040D000030001270006000500012300050005007C
:1040E00001550008000F000162000800120001B62F
:1040F000000D00220002010000000000013200005B
:1041000000000001F20156001E0102000000000044
:104110000001320000000000010C01E8FF30000245
:104120000100000000000132000000000001540006
:104130002100DAFF02000000000000013200000050
:10414000000001FF00EAFF2E000201000000000055
:1041500001320000000000019B00B4FFCAFF020012
:10416000000000000001320000000000011101E623
:10417000FF300002010000000000013200000000DA
:104180000001EC008A001F00020000000000000196
:10419000320000000000011C01E9FF3400020100B0
:1041A0000000000001320000000000017C00E6FF7A
:1041B000BAFF020000000000000132000000000011
:1041C00001C201A6FF01000201000000000001324F
:1041D0000000000000019C005C00F0FF02000000F5
:1041E0000000000132000000000001C701A5FF022D
:1041F0000002010000000000013200000000000188
:10420000E60068005B0002000000000000013200D0
:104210000000000001BD01A7FF0100020100000035
:104220000000013200000000000194005900FFFF6F
:104230000200000000000001320000000000018CBC
:1042400001F2FFB2FF020100000000000132000095
:10425000000000017C001900460002000000000080
:104260000001320000000000018701F2FFB3FF02ED
:104270000100000000000132000000000001CB003E
:10428000AAFF5600020000000000000132000000FA
:104290000000018E01F0FFB2FF02010000000000EB
:1042A0000132000000000001DD007400C0FF0200C8
:1042B00000000000000132000000000001BD01A765
:1042C000FF010002010000000000013200000000B8
:1042D00000019B004B0037000200000000000001BD
:1042E000320000000000014100F5FF07000201005C
:1042F0000000000001320000000000011700000073
:10430000F2FF020000000000000132000000000087
:10431000014600FFFF0E0002010000000000013214
:1043200000000000000119000100F1FF0200000080
:10433000000000013200000000000144000B0008F2
:104340000002010000000000013200000000000136
:10435000B60093FF010002000000000000013200DF
:104360000000000001350007000800020100000005
:10437000000001320000000000011B000200F0FFFD
:1043800002000000000000013200000000000139BE
:1043900000F7FF07000201000000000001320000EA
:1043A00000000001F2007B004D0002000000000050
:1043B0000001320000000000014400F5FF08000287
:1043C0000100000000000132000000000001A00018
:1043D000A0FFF9FF02000000000000013200000011
:1043E0000000018A01EFFFB3FF020100000000009E
:1043F00001320000000000015C001A00CFFF020043
:10440000000000000001320000000000011301E77D
:10441000FF31000201000000000001320000000036
:1044200000016D002200C8FF020000000000000132
:10443000320000000000013900F7FF070002010010
:10444000000000000132000000000001A400620032
:10445000F9FF02000000000000013200000000002F
:10446000014E0007000E00020100000000000132B2
:10447000000000000001D40086FF240002000000BC
:104480000000000132000000000001410000000DAA
:1044900000020100000000000132000000000001E5
:1044A0007700080047000200000000000001320011
:1044B00000000000013100070007000201000000B9
:1044C0000000013200000000000143026200B3FE60
:1044D0000200000000000001320000000000015155
:1044E00001F2FFBEFF0201000000000001320000E7
:1044F000000000016B0019003B00020000000000FA
:104500000001320000000000014B01F3FFBFFF0279
:104510000100000000000132000000000001450021
:10452000230016000200000000000001320000001D
:104530000000014B01F3FFBFFF020100000000007B
:104540000132000000000001FD009EFF7400020027
:10455000000000000001320000000000015501F3DE
:10456000FFBDFF020100000000000132000000005A
:10457000000118000300F2FF02000000000000012B
:1045800032000000000001FB001A00D5FF0201000C
:104590000000000001320000000000017B0030003C
:1045A000380002000000000000013200000000009E
:1045B000018101B3FF01000201000000000001328F
:1045C00000000000000186004F00F2FF0200000022
:1045D00000000001320000000000017C01B4FF0077
:1045E0000002010000000000013200000000000194
:1045F0007F004C00000002000000000000013200BB
:104600000000000001F4001700D5FF0201000000C7
:10461000000001320000000000015600F3FF3200EC
:10462000020000000000000132000000000001ED67
:10463000001600D6FF020100000000000132000059
:1046400000000001C400ECFF740002000000000044
:104650000001320000000000018101B3FF000002F0
:104660000100000000000132000000000001FD0018
:10467000580084FF0200000000000001320000002A
:104680000000016D01B7FF00000201000000000002
:104690000132000000000001E40049007400020043
:1046A00000000000000132000000000001ED0016D3
:1046B00000D6FF02010000000000013200000000EF
:1046C00000015B00D3FFE1FF0200000000000001D9
:1046D000320000000000013D000A00070002010056
:1046E0000000000001320000000000011600F4FF8D
:1046F000060002000000000000013200000000007F
:104700000143000C00FAFF0201000000000001322A
:104710000000000000011700F4FF07000200000085
:10472000000000013200000000000147000200F21A
:10473000FF02010000000000013200000000000143
:104740008500B1FF0D0002000000000000013200F2
:1047500000000000013E000300F4FF020100000021
:10476000000001320000000000017F0004004C0046
:1047700002000000000000013200000000000150B3
:1047800001F3FFBEFF020100000000000132000043
:104790000000000102000000FFFF02000000000016
:1047A00000013200000000000143000900F6FF0292
:1047B00001000000000001320000000000011600AE
:1047C000F7FF0A00020000000000000132000000B4
:1047D00000000124000600040002010000000000A7
:1047E00001320000000000010D00FAFFFBFF020093
:1047F0000000000000013200000000000102011B67
:1048000000D4FF020100000000000132000000009F
:10481000000102000000FFFF020000000000000194
:104820003200000000000135000800F9FF0201001D
:10483000000000000132000000000001CB00EBFF8F
:1048400078000200000000000001320000000000BB
:1048500001200005000400020100000000000132F8
:1048600000000000000182004E0000000200000075
:10487000000000013200000000000141000B00F9BF
:10488000FF020100000000000132000000000001F2
:10489000C30001008BFF0200000000000001320095
:1048A00000000000013900080008000201000000BB
:1048B00000000132000000000001AF0E3200CF08FE
:1048C00002010000000000013200000000000201AF
:0C48D000000000000000000000000000DC
:0448DC00E9CFE4FF3D
:1048E000EACFE4FFE652D9CFE6FFDACFE6FFE1CF29
:1048F000D9FFE2CFDAFFE6529EA0DFD29E908E0E65
:10490000CE6ECF6815C62CF606012D6B0601010E82
:104910002E6F0601165117111811191117E0D880C2
:10492000000E06011655000E1755190E1855000EEB
:10493000195506E20601166B176B186B196B06D03A
:1049400006011607000E175B185B195B060116516E
:1049500017111811191102E006012E6B060100054E
:1049600001E03DD106010D510E110F11101107E1AB
:104970000601115112111311141101E12FD1060179
:10498000C3510DE1060115A302D08C8E01D08C9E7F
:10499000060115A702D08C8A01D08C9A0FD006018F
:1049A000C3050CE1060115A302D08B8401D08B94C2
:1049B000060115A702D0898401D0899406010D5102
:1049C0000E110F11101164E0010EE96E060EEA6E71
:1049D0000E01B751EE240E01B76F0E01B851EE2053
:1049E0000E01B86F0E01B951EE200E01B96F0E0124
:1049F000BA51EE200E01BA6FD880000E0E01B755E5
:104A0000000EB855000EB955800EBA5529E2B7CE42
:104A1000B7FEB8CEB8FEB9CEB9FEBACEBAFE800E99
:104A20000E01BA5F010E06012C1106012C6F060162
:104A3000010E2D6F06010D07000E0E5B0F5B105B64
:104A4000060115A307D006012407000E255B265B8F
:104A5000275B06D00601242B000E252326232723BF
:104A600009C64CF00AC64DF04E6A4F6A4DAE02D0F0
:104A70004E684F684C50060101274D500601022335
:104A80004E50060103234F500601042306012E6BEE
:104A90000601115112111311141164E0050EE96E93
:104AA000060EEA6E0E01BB51EE240E01BB6F0E0125
:104AB000BC51EE200E01BC6F0E01BD51EE200E0167
:104AC000BD6F0E01BE51EE200E01BE6FD880000EEC
:104AD0000E01BB55000EBC55000EBD55800EBE55D7
:104AE00029E2BBCEBBFEBCCEBCFEBDCEBDFEBECE63
:104AF000BEFE800E0E01BE5F040E06012C110601E3
:104B00002C6F0601010E2D6F06011107000E125BBE
:104B1000135B145B060115A707D006012807000EDA
:104B2000295B2A5B2B5B06D00601282B000E29236C
:104B30002A232B230BC64CF00CC64DF04E6A4F6A4D
:104B40004DAE02D04E684F684C50060105274D50BF
:104B5000060106234E50060107234F500601082385
:104B600006012E6B06012D5139E00601C35107E104
:104B700006012CB18C8C06012CB58C8809D006015D
:104B8000C30506E106012CB18B8C06012CB5898A80
:104B90000000000000000000000000000000000015
:104BA0000000000000000000000000000000000005
:104BB00000000000000000000000000000000000F5
:104BC0000000000000000601C35103E18C9C8C989A
:104BD00005D00601C30502E18B9C899AD7D0030E4C
:104BE0000601005D01E0A0D00601D05101E179D0BD
:104BF00006011D05DF6E06011A511B1137E1DF505A
:104C0000EA6A310FE96E0E0EEA22EF500E01EA6AEF
:104C1000AC25E96EAD51EA22EF6AEA6ADF34FE0B99
:104C2000EA36E96E790EE9260E0EEA22EE6AED6AA0
:104C3000EA6ADF34FE0BEA36E96E490EE9260E0E0B
:104C4000EA22EE6AED6ADF50EA6A310FE96E0E0E73
:104C5000EA22EF6AEA6ADF34FE0BEA36E96E010EF9
:104C6000E9260E0EEA22EE6AED6A3BD0EA6ADF34EC
:104C7000FE0BEA36E96E790EE9260E0EEA221EC612
:104C8000EEFF1FC6EDFFEA6ADF34FE0BEA36E96E7F
:104C9000490EE9260E0EEA221AC6EEFF1BC6EDFFEC
:104CA000DF50EA6A310FE96E0E0EEA221CC6EFFFF2
:104CB000EA6ADF34FE0BEA36E96E010EE9260E0ED3
:104CC000EA22EE50ED100DE1EA6ADF34FE0BEA361F
:104CD000E96E010EE9260E0EEA221AC6EEFF1BC689
:104CE000EDFF0E01B65106011C5D1DE10E01B05134
:104CF00006011A1904E10E01B15106011B190AE15E
:104D00000601010EC46F0601C06B0601CF5101E020
:104D10008A9809D00601C46B0601010EC06F060116
:104D2000CF5101E08A8832D0040E0601005D2EE1E9
:104D30000601205124E021C64CF022C64DF0D89047
:104D40004D324C32D8904D324C324C50BB6ECDC6A9
:104D50004EF0CEC64FF0040ED8904E364F36E804D3
:104D6000FBE1300E4E16000E4F16CF0EBA140001A6
:104D70004E104C6E4FC04DF04C50BA6E04D0BB6A12
:104D8000CF0EBA14BA6E0601010E2E6F06012E5117
:104D900001E187D00601165117111811191101E010
:104DA00080D00601006B0601235176E130C600F683
:104DB00031C601F632C602F633C603F634C604F62F
:104DC00035C605F636C606F637C607F638C608F6FF
:104DD00039C609F63AC60AF63BC60BF63CC60CF6CF
:104DE0003DC60DF63EC60EF63FC60FF640C610F69F
:104DF00041C611F642C612F643C613F644C614F66F
:104E000045C615F646C616F647C617F648C618F63E
:104E100049C619F64AC61AF64BC61BF64CC61CF60E
:104E20004DC61DF64EC61EF64FC61FF650C620F6DE
:104E300051C621F652C622F60601306B0601316BCF
:104E4000326B336B346B0601356B366B376B386BFB
:104E500006013D6B3E6B3F6B406B0601416B426B45
:104E6000436B446B0601456B0601466B476B486B11
:104E7000496B06014A6B4B6B06014C6B06014D6B8F
:104E800006014E6B4F6B0601506B0601516B526B66
:104E90000601010E236F05D00601166B176B186B08
:104EA000196B8050800B06E00601CB5106E0815063
:104EB000010B03E10601010ECA6FE552E552E5CF91
:104EC000DAFFE7CFD9FFE552E5CFEAFFE5CFE9FF0B
:104ED0001100D9CFE6FFDACFE6FFE1CFD9FFE2CF6D
:104EE000DAFFE652DF6ADFCF00F0020EE76E00184D
:104EF000E8AE02D0E73402D0E750005C37E2DFCF03
:104F0000E9FFEA6AE9BEEA68D890E936EA36D8905D
:104F1000E936EA36010EE926060EEA22010EEE6EA9
:104F2000EE6AEE6AEE6ADFCFE9FFEA6AE9BEEA6896
:104F3000D890E936EA36D890E936EA360D0EE926F9
:104F4000060EEA22EE6AEE6AEE6AEE6ADFCFE9FF4B
:104F5000EA6AE9BEEA68D890E936EA36090EE92637
:104F6000060EEA22EE6AED6ADF2ABDD70601006B63
:104F70000601156B0601166B176B186B196B060192
:104F80001A6B1B6B06011C6B06011D6B06011E6B69
:104F90001F6B0601010E236FCD92CD9ECD9CCD8A55
:104FA000CD98CD96CD948E0ECE6ECF68CD809F805D
:104FB0009E909D8092809F9C010EE66EE66AA7EC13
:104FC0003DF0E552E552010EE66E0B0EE66EA7ECE3
:104FD0003DF0E552E5528D8496948D829692898CAF
:104FE000929C8D8096908B8294928C9C959C8C9EAA
:104FF000959E8C9895988C9A959A949E828E000096
:1050000000000000000000000000000000000000A0
:105010000000000000000000000000000000000090
:1050200000000000948E829E0601010ECF6F0601E3
:10503000010ED06F8A9893980601010EC06F060189
:10504000C36B0601010EC46F0601C96B0601C56B77
:10505000C66BC76BC86B0601CA6B9380F19E0601D5
:10506000010ECB6F939681964CEC32F0E552E552EF
:10507000E5CFDAFFE7CFD9FF120083EC32F0B6ECD0
:1050800033F06FEC33F0F9EC35F0E66AD950E6EC2A
:1050900035F00701B45101E0B3D0DF0424E1BFECE7
:1050A00033F00CE10601010ECF6FD06B94EC33F0BE
:1050B00002E2E16AE552E16E00500DD032EC34F0CC
:1050C00006E1ED5004E10601CF6B010E03D00601AD
:1050D000010ECF6FD06F000EE66EE66AC4C6E6FF23
:1050E0006BEC34F08BD0020EDF5C2EE1BFEC33F0C2
:1050F00009E10601C36B96909492959C959E9598B4
:10510000959A1BD032EC34F00DE1ED500BE1060125
:10511000010E79EC34F094949294949C929A959226
:1051200092926CD0D1EC35F0020EEE1867E1ED50A2
:1051300065E10601020E79EC34F094849284948C3B
:10514000928A958292825AD0040EDF5C07E1010EAA
:10515000DBCFB0FE020EDBCFB1FE50D0050EDF5C20
:1051600007E1010EDBCFAEFE020EDBCFAFFE46D075
:10517000080EDF5C0FE1D1EC35F0180ED880EE544C
:10518000000EED5403E2180E85EC34F0010EDBCF77
:10519000AAFE34D0090EDF5C0FE1D1EC35F0060E2B
:1051A000D880EE54000EED5403E2060E85EC34F088
:1051B000010EDBCFABFE22D00A0EDF5C03E18CECEC
:1051C00034F009D00B0EDF5C03E18CEC34F016D028
:1051D0000C0EDF5C07E1010EDBCFB4FE020EDBCF6D
:1051E000B5FE0CD00D0EDF5C09E1BFEC33F004E03E
:1051F0000601010ECB6F02D00601CB6B0EEC3DF029
:10520000E2EC35F0ABEF32F083EC32F0200EE1242B
:1052100002E3E168E65289EC35F036EC34F0E66AF8
:10522000D950040F14EC33F074EC35F0060F14EC85
:1052300033F074EC35F0080FF9EC34F0E66AD9502D
:105240000C0FF9EC34F0D950040F1EEC34F004E2EA
:10525000F80E006EB00E7FD2D950060F1EEC34F05F
:1052600004E2CA0E006EB00E76D210EC34F0040EDA
:10527000005C000E015804E2A00E006EB00E6BD26E
:10528000060EDBCF00F0070EDBCF01F0040E005C52
:10529000000E015804E2780E006EB00E5CD20701D9
:1052A000B45101E061D2080EDBCF10F0090EDBCF64
:1052B00011F00A0EDBCF12F00B0EDBCF13F010C093
:1052C00038F011C039F012C03AF013C03BF0080EAC
:1052D000DBCF3DF0090EDBCF3EF00A0EDBCF3FF017
:1052E0000B0EDBCF40F017EC63F034C00CF035C090
:1052F0000DF036C00EF037C00FF00C0EDBCF14F0FF
:105300000D0EDBCF15F00E0EDBCF16F00F0EDBCF40
:1053100017F014C038F015C039F016C03AF017C0B5
:105320003BF00C0EDBCF3DF00D0EDBCF3EF00E0E52
:10533000DBCF3FF00F0EDBCF40F017EC63F00C50EB
:105340003424086E0D503520096E0E5036200A6E3A
:105350000F5037200B6E17EC34F03B6E0AEC54F014
:1053600019EC33F039C0E6FF3AC0E6FF3BC0E6FF78
:105370003CC0E6FF87EC59F0E2EC35F0E55297ECE3
:1053800035F038C039F0B9EC35F07AEC55F0140E40
:1053900038C0DBFF150E39C0DBFF160E3AC0DBFF4D
:1053A000170E3BC0DBFF06012351FDE03FEC34F05C
:1053B000080FE96E000E5FEC33F002E666EC33F0A6
:1053C00010E2020E456FC2EC34F0080E34C0DBFF71
:1053D000090E35C0DBFF0A0E36C0DBFF0B0E37C0EF
:1053E000DBFFD9500C0FE96E000E5FEC33F002E6E4
:1053F00066EC33F012E2080E06014511456F0C0E03
:10540000DBCF38F00D0EDBCF39F00E0EDBCF3AF0EC
:105410000F0EE3EC32F045EC33F0CEEC34F002E664
:10542000EDEC32F004E24A0E006EB00E94D1DAECEC
:1054300034F002E6EDEC32F004E21C0E006EB00E29
:105440008AD1C3EC33F019EC33F0AC0E3E6EC50ECE
:105450003F6EA70E406E470E416E76EC54F025EC81
:1054600034F0DBCF0CF0150EDBCF0DF0160EDBCFDA
:105470000EF0170EDBCF0FF00CC038F00DC039F076
:105480000EC03AF00FC03BF008EC54F048EC34F09A
:10549000D8EC32F023EC54F0180E39C0DBFF190EB3
:1054A0003AC0DBFF1A0E3BC0DBFF1B0E3CC0DBFF2C
:1054B000EAEC33F0080EDBCF08F0090EDBCF09F081
:1054C0000A0EDBCF0AF00B0EFDEC34F038C031F6DB
:1054D00039C032F63AC033F63BC034F6080EDBCFA3
:1054E0003DF6090EDBCF3EF60A0EDBCF3FF60B0E84
:1054F000DBCF40F651EC34F048EC34F051EC34F0B2
:1055000039C00CF03AC00DF03BC00EF03CC00FF0BB
:10551000B4EC34F008C039F009C03AF00AC03BF0EE
:105520000BC03CF076EC54F019EC33F0C3EC33F0E4
:1055300039C014F03AC015F03BC016F03CC017F06B
:10554000C3EC33F039C018F03AC019F03BC01AF080
:105550003CC01BF0B4EC34F014C039F015C03AF084
:1055600016C03BF017C03CF076EC54F039C010F098
:105570003AC011F03BC012F03CC013F0B4EC34F070
:1055800004C039F005C03AF006C03BF007C03CF05B
:10559000E3EC54F025EC34F0DBCF28F0150EDBCF34
:1055A00029F0160EDBCF2AF0170EDBCF2BF028C028
:1055B00038F029C039F02AC03AF02BC03BF008EC93
:1055C00054F039C024F03AC025F03BC026F03CC06E
:1055D00027F0140EDBCF30F0150EDBCF31F0160EB6
:1055E000DBCF32F0170EDBCF33F030C038F031C0F4
:1055F00039F032C03AF033C03BF008EC54F039C017
:105600002CF03AC02DF03BC02EF03CC02FF0B4EC93
:1056100034F024C039F025C03AF026C03BF027C052
:105620003CF076EC54F039C020F03AC021F03BC099
:1056300022F03CC023F03E6A3F6A406A400E416E51
:1056400076EC54F039C01CF03AC01DF03BC01EF09F
:105650003CC01FF0D8EC32F023EC54F01C0E39C0E3
:10566000DBFF1D0E3AC0DBFF1E0E3BC0DBFF1F0E33
:105670003CC0DBFF080EDBCF04F0090EDBCF05F0EA
:105680000A0EDBCF06F00B0EB1EC32F038C039F663
:1056900039C03AF6EAEC33F00C0EDBCF08F00D0E11
:1056A000DBCF09F00E0EDBCF0AF00F0EFDEC34F06D
:1056B00038C035F639C036F63AC037F63BC038F652
:1056C0000C0EDBCF41F60D0EDBCF42F60E0EDBCF1C
:1056D00043F60F0EDBCF44F6A9EC34F0B1EC32F018
:1056E00038C03BF639C03CF610EC34F0060EDB5007
:1056F000001803E1070EDB50011812E006013951D2
:105700003A110EE1D880000E3D55000E3E55000EB8
:105710003F55000E405504E2F10E006EAF0E1BD057
:1057200010EC34F0060EDB50001803E1070EDB50DE
:10573000011814E006013B513C1110E1D880000E25
:105740004155000E4255000E4355000E445506E2E9
:10575000C60E006EAF0E14EC35F006D00601010E39
:10576000306F236B0EEC3DF0200EE15C02E2E16A4B
:10577000E552E16EABEF32F083EC32F0100EE12433
:1057800002E3E168E65289EC35F06FEC33F074EC3B
:1057900035F0040FF9EC34F081EC34F0080FF9EC3B
:1057A00034F00E01BF516FE0DDEC32F002E1070191
:1057B000B48D0701B45173E1DFEC33F004E2930ED2
:1057C000006EAF0E5DD020EC35F002E640EC33F019
:1057D00005E2D950040F78EC33F004D02CEC35F00E
:1057E00045EC33F0DAEC34F002E6EDEC32F004E2B2
:1057F0004A0E006EB00E44D038EC35F004E2630E71
:10580000006EAF0E3DD05FEC32F00C0FF7EC32F0D3
:1058100009E3A9EC34F022EC33F004E03D0E006E15
:10582000AF0E2ED0CEEC34F002E640EC33F005E2C1
:10583000D950080F78EC33F004D0C2EC34F045ECCA
:1058400033F0DAEC34F002E6EDEC32F004E21C0E58
:10585000006EB00E15D038EC35F004E20D0E006E7F
:10586000AF0E0ED05FEC32F00C0FF7EC32F00BE322
:10587000A9EC34F022EC33F006E0E70E006EAE0E39
:1058800014EC35F00CD00AEC35F002E2E16AE55296
:10589000E16E00500701E35102E00EEC3DF0100E06
:1058A000E15C02E2E16AE552E16EABEF32F083ECDB
:1058B00032F0180EE12402E3E168E65289EC35F09B
:1058C00036EC34F0140EDB6A150EDB6A160EDB6A5A
:1058D000170EDB6A6FEC33F074EC35F00C0FF9EC5B
:1058E00034F0E66AD950100FF9EC34F0DDEC32F008
:1058F00002E10701B48D100EDBCF00F0110EDBCFFB
:1059000001F0120EDBCF02F0130EDBCF03F0D95003
:105910000C0FBDEC34F0EE500026EE500122EE509C
:105920000222EE500322040E00C0DBFF050E01C070
:10593000DBFF060E02C0DBFF070E03C0DBFFA9EC96
:1059400034F0DBCF07F0D950100FBDEC34F0EE503F
:10595000045C006EEE500558016EEE500658026E63
:10596000EE500758036E080E00C0DBFF090E01C0A1
:10597000DBFF0A0E02C0DBFF0B0E03C0DBFF20ECD7
:1059800035F002E640EC33F005E2D950040F86EC26
:1059900033F004D02CEC35F0F7EC33F0DFEC33F0DF
:1059A00004E2930E006EAF0E4AD044EC35F002E6EE
:1059B000EDEC32F004E24A0E006EB00E40D050EC36
:1059C00035F004E2630E006EAF0E39D05FEC32F0BA
:1059D000140FF7EC32F007E35CEC35F004E03D0E19
:1059E000006EAF0E2CD0CEEC34F002E640EC33F07B
:1059F00005E2D950080F86EC33F004D0C2EC34F045
:105A0000F7EC33F044EC35F002E6EDEC32F004E272
:105A10001C0E006EB00E13D050EC35F004E20D0EEB
:105A2000006EAF0E0CD05FEC32F0140FF7EC32F0DA
:105A300009E35CEC35F006E0E70E006EAE0E14EC08
:105A400035F00CD00701B45109E10AEC35F002E25F
:105A5000E16AE552E16E00500EEC3DF0180EE15C9B
:105A600002E2E16AE552E16EABEF32F0F5EC35F0BF
:105A7000DE6A72EC33F006012351FDE07EEC35F076
:105A8000CBEC33F026E168EC35F023E1020E306F09
:105A9000FA0EDBCF46F6FB0EDBCF47F6FC0EDBCF74
:105AA00048F6FD0EDBCF49F6D9EC33F046C638F0A8
:105AB00047C639F048C63AF049C63BF017EC63F0E8
:105AC00034C046F635C047F636C048F637C049F60A
:105AD00010D13FEC34F0F60FB5EC35F002E666EC91
:105AE00033F01BE2020E4511456FF60EDBCF38F0A6
:105AF000F70EDBCF39F0F80EDBCF3AF0F90EE3EC1E
:105B000032F0F60E34C0DBFFF70E35C0DBFFF80EC7
:105B100036C0DBFFF90E37C0DBFFD950F20FB5EC12
:105B200035F002E666EC33F01CE2080E0601451182
:105B3000456FF20EDBCF38F0F30EDBCF39F0F40E09
:105B4000DBCF3AF0F50EE3EC32F0F20E34C0DBFFBF
:105B5000F30E35C0DBFFF40E36C0DBFFF50E37C0A9
:105B6000DBFFD950F60FB5EC35F002E659EC34F016
:105B70000DE20F0E006ED950F60FA3EC33F003E0E8
:105B8000D2EC33F0FDE1C0EC35F009D07EEC35F01D
:105B9000D5EC35F0D2EC33F0FDE1D9EC33F029EC63
:105BA00033F00CE2EBEC32F0B20E006EAE0E79EC9C
:105BB00035F002E2E16AE55228EC34F0DDEC32F037
:105BC00012E1F60EDBCF04F0F70EDBCF05F0F80E96
:105BD000DBCF06F0F90E22EC33F005E0870E006E05
:105BE000AE0EEBEC35F0B2EC33F003E093EC34F0B6
:105BF000FDE104EC34F0DFCF31F6010EDBCF32F6FD
:105C0000020EDBCF33F6030EDBCF34F6F60EDBCF1E
:105C10003DF6F70EDBCF3EF6F80EDBCF3FF6F90E82
:105C2000DBCF40F60601396B3A6BD950F20FB5EC79
:105C300035F002E659EC34F00DE20F0E006ED9504B
:105C4000F20FA3EC33F003E0D2EC33F0FDE1C0EC53
:105C500035F011D0F20EDBCF00F0F30EDBCF01F008
:105C6000F40EDBCF02F0F50ED5EC35F0D2EC33F0CC
:105C7000FDE1D9EC33F029EC33F00CE2EBEC32F03F
:105C8000520E006EAE0E79EC35F002E2E16AE5529A
:105C900028EC34F0DDEC32F008E168EC35F005E09A
:105CA000270E006EAE0EEBEC35F0B2EC33F003E0F5
:105CB00093EC34F0FDE104EC34F0DFCF35F6010E67
:105CC000DBCF36F6020EDBCF37F6030EDBCF38F62E
:105CD000F20EDBCF41F6F30EDBCF42F6F40EDBCF54
:105CE00043F6F50EDBCF44F606013B6B3C6B010E31
:105CF000306F0601236B040EE15C02E2E16AE552BB
:105D0000E16EABEF32F083EC32F0110EE12402E3EE
:105D1000E168E65262EC34F092EC32F0100EDB6A8D
:105D20000601235102E1300502E0000502E1010E07
:105D3000DF6E300527E1306B090E3DC6DBFF0A0E32
:105D40003EC6DBFF0B0E3FC6DBFF0C0E40C6DBFF83
:105D50000D0E41C6DBFF0E0E42C6DBFF0F0E43C623
:105D6000DBFF100E44C6DBFF3D6B3E6B3F6B406BB1
:105D7000416B426B436B446B396B3A6B3B6B3C6BD7
:105D8000010E236F000525E1006B010E0DC6DBFF40
:105D9000020E0EC6DBFF030E0FC6DBFF040E10C69D
:105DA000DBFF050E11C6DBFF060E12C6DBFF070E7A
:105DB00013C6DBFF080E14C6DBFF0D6B0E6B0F6BFB
:105DC000106B116B126B136B146B096B0A6B0B6B03
:105DD0000C6BD950050F95DBD950010F92DBD950D0
:105DE0000D0F8FDBD950090F8CDBDFCFE6FFE66AA2
:105DF000120E006EAE0E8DDB036E150EE15C02E23C
:105E0000E16AE55275EC34F0110EE15C02E2E16A00
:105E1000E552E16EA0D3C4C600F0016A00BE01687D
:105E20009AEC34F00D0E026EAE0E52EC33F002E23C
:105E3000E16AE552E16E05500EEF3DF017EC35F0EA
:105E4000DE6ADD6A010EE66ECCEC35F0030E31DB66
:105E50000701B4510FE10601C40504E19FEC34F0E1
:105E6000E66A04D09FEC34F0010EE66E6BEC34F081
:105E70000EEC3DF0E552E5526ED317EC35F0B6EC82
:105E800033F06FEC34F01BEC35F0A0EC35F0A4EC03
:105E900034F00701B45129E1030EDB50070802E298
:105EA0006FEC34F0DF50010802E2010EDF6E030EEA
:105EB000DB50030F0E01B65D0CE094EC33F002E210
:105EC000E16AE552E16E0050030EDB50030F0E0154
:105ED000B66F010EDBCFE6FF020EDBCFE6FFDFCFB2
:105EE000E6FF6BEC34F00EEC3DF0050EE15C02E2F7
:105EF000E16AE552E16E2FD3F5EC35F0FD0EDB04DF
:105F00000BE1B0CEDEFFB1CEDDFF020EB2CEDBFF85
:105F1000030EB3CEDBFF0AD0AECEDEFFAFCEDDFF89
:105F2000020EB4CEDBFF030EB5CEDBFFFB0EDBCFE4
:105F3000E6FFFC0EDBCFE6FF020EDBCFE6FF030E33
:105F4000DBCFE6FFB6CEE6FF9FEC34F072EC5EF0FE
:105F5000006E070EE15C02E2E16AE552E16E00507C
:105F6000040EE15C02E2E16AE552E16EF4D217EC64
:105F700035F0E652B4DBA5EC35F039E10701B45158
:105F800056E10601C35103E0020EC35D28E1DF5074
:105F9000000821E2C35101E18D90DF0403E18D840B
:105FA0008D82898C020EDF5C03E18D848D82899C59
:105FB000030EDF5C03E18D948D82899C040EDF5C0F
:105FC00003E18D848D92899C050EDF5C10E18D9438
:105FD0008D92899C0CD0C3510AE18D8008D0C305F5
:105FE00006E1DF50000802E28C9201D08C8281EC45
:105FF00034F0010F19DBA5EC35F017E10701B451BE
:1060000016E10601C35108E1010EDB50000802E26F
:106010008B920BD08B8209D0C30507E1010EDB50B8
:10602000000802E2899201D089820EEC3DF0E2EC98
:1060300035F091D2FE0E0601C55DFF0EC659FF0E6A
:10604000C759FF0EC85905E2C52B000EC623C7234A
:10605000C8230EEF3DF00601C551C611C711C81186
:1060600005E0C507000EC65BC75BC85B0EEF3DF0E1
:10607000F5EC35F0E65233DB070E1BDAA4EC34F016
:10608000DB500BE1DFCFC5F6010EDBCFC6F6020E0B
:10609000DBCFC7F6030EDBCFC8F60EEC3DF0050EE6
:1060A000E15C02E2E16AE552E16E55D2C5C6E6FF67
:1060B000C6C6E6FFC7C6E6FFC8C6E6FF040E006E0A
:1060C000AE0E79EC35F002E2E16AE55275EF34F09C
:1060D000E66AC90EE66E060EE66EF9EC35F00701CB
:1060E000B45101E012000EEF3DF0C9C600F0016AA4
:1060F00000BE01689AEC34F0FD0E026EAD0ED2DAED
:1061000002E2E16AE552E16E05500EEF3DF0CAC6CB
:1061100000F0016A00BE01689AEC34F0F70E026EDE
:10612000AD0EC0DA02E2E16AE552E16E0550060109
:10613000CA6B0EEF3DF09DBCFED716C1E6FF17C13E
:10614000E6FF00C1E6FF01C1E6FFEB0E006EAD0EFB
:1061500079EC35F002E2E16AE55275EF34F017ECC4
:1061600035F004DB030EDB6A1BEC35F0EDDBA0EC55
:1061700035F00701B45101E080D0D1EC35F0FF0ECD
:10618000D880EE54030EED5407E2010EDB68030ED7
:10619000F36E020EF3CFDBFFDF50010802E2010EC7
:1061A000DF6E030EDB50010801E299DBDF0409E139
:1061B000040EDB50030805E10601CD6B020ECE6F25
:1061C00006D0010EDBCFCDF6020EDBCFCEF6CAB481
:1061D00015D0CB68FC0ECA140009CA6E9D920F013F
:1061E00052815293F00EBA140C09BA6E3F0EBA14D3
:1061F0000009BA6E0E010E0ECC6FCA84030EDB507E
:106200002AE1DF5023E0CDC600F0CEC601F0D890E1
:1062100001320032D890013200320050BB6ECDC640
:1062200002F0CEC603F0040ED89002360336E8041E
:10623000FBE1300E0216000E0316CF0EBA14000159
:106240000210006E03C001F0E85003D0BB6ACF0E0D
:10625000BA14BA6E10D006012351FDE0CDC651F636
:10626000CEC652F6466B476B486B496BDFCF50F694
:10627000040E306F236B0EEC3DF0050EE15C02E284
:10628000E16AE552E16E67D112003DD9270EE124A3
:1062900002E3E168E65216DBF29E040E00C6DBFF65
:1062A000050E01C6DBFF060E02C6DBFF070E03C6A6
:1062B000DBFF080E04C6DBFF090E05C6DBFF0A0E76
:1062C00006C6DBFF0B0E07C6DBFF0C0E08C6DBFFA6
:1062D0000D0E09C6DBFF0E0E0AC6DBFF0F0E0BC646
:1062E000DBFF100E0CC6DBFF110E0DC6DBFF120E1E
:1062F0000EC6DBFF130E0FC6DBFF140E10C6DBFF4E
:10630000150E11C6DBFF160E12C6DBFF170E13C6E5
:10631000DBFF180E14C6DBFF190E15C6DBFF1A0EC5
:1063200016C6DBFF1B0E17C6DBFF1C0E18C6DBFFF5
:106330001D0E19C6DBFF1E0E1AC6DBFF1F0E1BC685
:10634000DBFF200E1CC6DBFF210E1DC6DBFF220E6D
:106350001EC6DBFF230E1FC6DBFF240E20C6DBFF9D
:10636000250E21C6DBFF260E22C6DBFFF28E1A0E9B
:10637000DBCF00F01B0EDBCF01F01C0EDBCF02F0F9
:106380001D0E09DA02E0010EDF6E040EDB5002E0A2
:10639000010EDF6E0601235106E1010EDF6EF36E82
:1063A000030EF3CFDBFFDF500FE0110EDBCF00F069
:1063B000120EDBCF01F0130EDBCF02F0140EEBD97F
:1063C00003E0DE52010EDD6EDF5011E0150EDBCF73
:1063D00000F0160EDBCF01F0170EDBCF02F0180E27
:1063E000DAD905E0010EF36E020EF3CFDBFF030EE8
:1063F000DBCFE6FFE66A020EDBCFE6FFE66A010EC0
:10640000DBCFE6FFE66ADFCFE6FFE66ADA0E006E74
:10641000AD0E7FD8036E0B0EE15C02E2E16AE5523D
:10642000E16E0350270EE15C02E2E16AE552E16EA3
:1064300092D069D8080EE12402E3E168E652E16EE9
:10644000F29E24C6DFFF010E25C6DBFF020E26C624
:10645000DBFF030E27C6DBFF040E28C6DBFF050E9D
:1064600029C6DBFF060E2AC6DBFF070E2BC6DBFFA5
:10647000F28EB6DBD00E006EAD0E4BD8036E0B0E57
:10648000E15C02E2E16AE55230DA080EE15C02E228
:10649000E16AE552E16E5FD0F29E0601246B256B46
:1064A000266B276B286B296B2A6B2B6BF28E0EEFFA
:1064B0003DF0E66E6DEC42F085DBE552120086DAC7
:1064C0001F0E3D6E050E3E6E3F6A406A89DA75EC1E
:1064D00063F02DDBD9501200DBCF03F081DADFCF80
:1064E0003DF0010EDBCF3EF0020EDBCF3FF0030E9E
:1064F000DBCF40F075EC63F0D880190E3854C5EF4F
:1065000035F03BDA0BD348DBE1CFD9FFE2CFDAFF3E
:106510001200016E026A00C0E6FFE66E02C0E6FFEE
:1065200041EF62F0040EDB6A050EDB6A060EDB6AE1
:10653000070EDB6A080EDB6A090EDB6A0A0EDB6AED
:106540000B0EDB6A0C0EDB6A0D0EDB6A0E0EDB6ACD
:106550000F0EDB6A1200E552E5CFDAFFE7CFD9FF75
:106560001200DBCF07F004C038F005C039F006C0D8
:106570003AF007C03BF00AEC54F01C0EDBCF3EF0C3
:106580001D0EDBCF3FF01E0EDBCF40F01F0EDBCF2A
:1065900041F076EC54F0E0DA210E3E6EE60E3F6EEE
:1065A0005B0E406E400E416E76EC54F07AEF55F083
:1065B000DBD900C039F0B9EF35F008DA005001102E
:1065C000021003101200DBCF3BF03D683E683F68CD
:1065D000406817EF63F0F1DAA1D2D880FF0E39548A
:1065E000FF0E3A54FF0E3B54000E3C541200C5D926
:1065F000EE50385CEE503958EE503A58EE503B5859
:106600001200FA0EDBCF3DF0FB0EDBCF3EF0FC0EAE
:10661000DBCF3FF0FD0EDBCF40F01200DBCF3CF0D4
:106620003C34000E3C181200E66E000EDA20E66ED6
:10663000120039C004F03AC005F03BC006F03CC07F
:1066400007F01200DBCF07F004500510061007100A
:10665000120075EC63F038C0DEFF39C0DEFF3AC0CF
:10666000DEFF3BC0DDFFDD52DD52A7DAD880000E31
:10667000EE54800EEE54000EEE54000EEE54120056
:10668000D88083DA000E3C5412000C0E34C0DBFFBD
:106690000D0E35C0DBFF0E0E36C0DBFF0F0E37C010
:1066A000DBFF1200036E046A02C0E6FFE66E04C060
:1066B000E6FF41EC62F0056E050EE15C1200DA20A7
:1066C000EA6ED890030EEB50000A1200000EEE5C4A
:1066D000000EEE58000EEE58000EEE581200E66A5C
:1066E000CCEF35F0DE6ADE6ADD6ADD52DD52120083
:1066F00044D90C0EEECFDBFF0D0EEECFDBFF0E0EFE
:10670000EECFDBFF0F0EEECFDBFF120036D9140EFB
:10671000EECFDBFF150EEECFDBFF160EEECFDBFF6D
:10672000170EEECFDBFF1200000EE66EE66AE66E95
:10673000E66AB6CEE6FFE66EE66A72EC5EF0006EE2
:10674000070EE15C1200E96EFF0EDA20EA6E0050DF
:106750001F0BEECF38F0EECF39F0EECF3AF0EECFA0
:106760003BF0120033D9100E1F0B1200E652E65216
:10677000E652DF6A010EDB6A020EDB6A120011DAF2
:10678000EE50ED101200040EDBCF3AF0050EDBCF19
:106790003BF0F3EF53F0DBCF03F000500110021099
:1067A00003101200D890383639363A363B36E806B0
:1067B0001200190E3D6E3E6A3F6A406A1200FDD912
:1067C000D880FF0EEE54FF0EEE54FF0EEE54000E76
:1067D000EE541200180EDBCF00F0190EDBCF01F0E3
:1067E0001A0EDBCF02F01B0EDBCF03F01200140EEB
:1067F00034C0DBFF150E35C0DBFF160E36C0DBFFE5
:10680000170E37C0DBFF120000C0DFFF010E01C012
:10681000DBFF020E02C0DBFF030E03C0DBFF120032
:10682000040EDBCF00F0050EDBCF01F0120008C034
:1068300038F009C039F00AC03AF012009ED8A80E0C
:10684000D880EE54610EED54120086D9140E120059
:10685000E16E0350DE6A800EDE6EDE6ADD6ADD52B6
:10686000DD5212009ED9010EEE181200100EDB6AE6
:10687000110EDB6A120EDB6A130EDB6A1200466B26
:10688000476B486B496B456B8D908B92D9501200CA
:1068900039C008F03AC009F03BC00AF03CC00BF028
:1068A0001200060EDBCF3AF0070EDBCF3BF0F3EF22
:1068B00053F0FF0EEE5CFF0EEE58010EEE58000E88
:1068C000EE581200E16EDF6A010EDB6A020EDB6A2F
:1068D000030EDB6A12007CEC2FF0E2EF35F0010EC4
:1068E000F36E030EF3CFDBFF1200E16E03500EEFE9
:1068F0003DF0C36F96809482958C958E9588958A8D
:106900001200010EE66ED9501200F36E010EF3CFA5
:10691000DBFF020EDB6A1200010EDBCFB2FE020EBD
:10692000DBCFB3FE1200D8900036013602360336B4
:10693000E806120000C0E6FF01C0E6FF1200DECF4D
:10694000E6FFDDCFE6FF1200E76E040EE7CFDBFFC8
:1069500012000C0EDBCF04F00D0EDBCF05F00E0E97
:10696000DBCF06F00F0E120039C03EF03AC03FF008
:106970003BC040F03CC041F01200E96E000EDA204E
:10698000EA6E1200080EDBCF38F0090EDBCF39F0CB
:106990000A0EDBCF3AF00B0EE3EF32F0080EDBCF3E
:1069A00039F0090EDBCF3AF00A0EDBCF3BF00B0ECD
:1069B0000EEF33F00C0EDBCF39F00D0EDBCF3AF0DB
:1069C0000E0EDBCF3BF00F0E0EEF33F0F6D8EECF0E
:1069D00000F0EECF01F0EECF02F0EFCF03F01200A7
:1069E00000C038F001C039F002C03AF003C03BF0FB
:1069F00012001ADE060E59EF32F0DBCF0BF017DF74
:106A00000BC03BF00AEC54F014DED2DD76EC54F00F
:106A10007AEF55F0D950080F74DDE2D836EC2DF03E
:106A2000006E0C0EE15C120074DDE2EF35F06BDD00
:106A3000E652E652120053DEDCD863DFE6EF35F0B3
:106A4000040EDBCF39F0050EDBCF3AF0060EDBCFBC
:106A50003BF0070E0EEF33F0040EDBCF38F0050EDF
:106A6000DBCF39F0060EDBCF3AF0070EE3EF32F062
:106A70000C0EDBCF00F00D0EDBCF01F00E0EDBCFE6
:106A800002F00F0E6CEF32F0140EDBCF39F0150E62
:106A9000DBCF3AF0160EDBCF3BF0170E0EEF33F0E4
:106AA000140EDBCF00F0150EDBCF01F0160EDBCF9E
:106AB00002F0170E6CEF32F0140EDBCF04F0150E5F
:106AC000DBCF05F0160EDBCF06F0170E22EF33F00A
:106AD000F20EDBCF04F0F30EDBCF05F0F40EDBCFCC
:106AE00006F0F50E22EF33F0070EE3DCE66AD9502C
:106AF00012000FDD036E070EE15C1200F60EDBCF15
:106B000000F0F70EDBCF01F0F80EDBCF02F0F90E4C
:106B10001200E16EDE6AE6DD92EF32F0EECFE6FFC4
:106B2000EECFE6FFEECFE6FFEFCFE6FF120038C074
:106B300000F039C001F03AC002F03BC003F012008F
:106B4000E0DE030F71DDF9EF35F053D8E76E020E8A
:106B5000E7CFDBFFDB50120039C000F03AC001F094
:106B60003BC002F03CC003F01200E96EFF0E5FEF85
:106B700033F001C03AF002C03BF003C03CF0120019
:106B800018DE75EC63F001EF33F0000E3954000E9F
:106B90003A54000E3B541200D9CFE6FFDACFE6FF9D
:106BA0001200D950010FBDEF34F0DBCF03F018DF36
:106BB00028DD75EC63F00F0E1200D9CFE9FFDACFB4
:106BC000EAFF1200E552E552E5521200010F2CDDFA
:106BD000030E59EF32F028DF010EDE6E72EF33F054
:106BE000D950040F8EDCEBEF32F021DFE652E65293
:086BF0001200010E59EF32F012
:086BF800D8CFE4FFE0CFE4FF79
:106C0000E46EE9CFE4FFEACFE4FFF3CFE4FFF4CF93
:106C1000E4FFE65266EC46F0CBEC45F0030EDB6A8F
:106C2000A4A69ED1A4960E01002B0E01AB510E011D
:106C3000005D01E284D0006B0E0196EC45F0EF6A36
:106C400079907B6A7A6A0E01A92B0E01AA510E0176
:106C5000A95D01E3A96B5EEC46F0EA22EE50ED106F
:106C60006EE000EC47F0B0EC46F002E14B50491802
:106C700047E074EC46F0EA22EE50ED103AE08AEC80
:106C800046F071EC45F05EEC46F0EA22EE504A5CCC
:106C9000486EEE504B58496E020E48C0DBFF030EA3
:106CA00049C0DBFFEAEC45F0493412E248500008E5
:106CB000000E49540DE2EAEC45F074EC46F09AEC13
:106CC00046F017E2E7EC46F0EE264950ED2218D0E8
:106CD000EAEC45F0486C491E000E492274EC46F07F
:106CE0009AEC46F006E2E7EC46F0EE5E4950ED5ACB
:106CF00007D000EC47F0EA2248C0EEFF49C0EDFFA4
:106D000096EC45F0120EEF6EF29E0E015EEC46F030
:106D10002DEC45F049C048F0496A4850B66E5EEC2B
:106D200046F02DEC45F04850B56EF00EB414000955
:106D3000B46EF00EB4140909B46E7980F28E0701B6
:106D4000000ED880AA55000EAB552EE2B82B000ECF
:106D5000B923AA51B85DAB51B95926E3B86BB96BE9
:106D6000030EAE5D1FE2AC51EA6A200FE96E010E20
:106D7000EA2280CFEFFFAC51EA6A230FE96E010EE1
:106D8000EA2281CFEFFFAC51EA6A260FE96E010ECD
:106D9000EA2282CFEFFFAC2B030EAC5D01E3AC6BBC
:106DA000AE2B02D0AA6BAB6B000ED880AF55000E95
:106DB000B0551CE2000ED880BE55000EBF5516E23D
:106DC000BA2B000EBB23AF51BA5DB051BB590EE3D5
:106DD000BA6BBB6B030EB35D07E2B12B030EB15D63
:106DE00001E3B16BB32B02D0AF6BB06BBE51BF11DF
:106DF0000BE0050EBD5D07E3C18C9E9C9D8CC2809F
:106E0000C282BD6B01D0BD2B0501005101E1A4D0B0
:106E1000DE6ADD6ADECF48F0DDCF49F0040E485C63
:106E2000000E495801E398D033EC45F077EC45F07B
:106E3000FDE1010EE926050EEA22EE50ED1070E0AC
:106E400033EC45F077EC45F0FDE1B4EC46F0EE5064
:106E5000ED1016E1B9EC46F001E18180BDEC46F0A1
:106E600003E1ED5001E18182C1EC46F003E1ED5018
:106E700001E18184C5EC46F003E1ED5001E181863A
:106E800033EC45F077EC45F0FDE194EC46F077EC1F
:106E900045F0FDE1010EE926050EB0EC46F019E1E2
:106EA0004B50491816E1B9EC46F001E18190BDEC78
:106EB00046F003E1ED5001E18192C1EC46F003E1BF
:106EC000ED5001E18194C5EC46F003E1ED5001E1A4
:106ED000819633EC45F077EC45F0FDE1B4EC46F0FB
:106EE000EE2A000EEF2233EC45F077EC45F0FDE1A1
:106EF00094EC46F077EC45F0FDE1090EE926050E2D
:106F0000B0EC46F023E14B50491820E133EC45F05A
:106F100077EC45F0FDE1B4EC46F0EE6AED6A16D090
:106F2000B9EC46F001E18190BDEC46F003E1ED5093
:106F300001E18192C1EC46F003E1ED5001E1819461
:106F4000C5EC46F003E1ED5001E18196DF2A010E28
:106F500001E260D7DB2A5ED70601CC5101E0CC0705
:106F60009EAC3DD09E9CC1AC07D0C19C010E0701D8
:106F7000C06FC16BBC6B18D0C4504A6E4B6E4A6A6E
:106F8000C35000014A10486E4BC049F00701BC5184
:106F9000E96EEA6ABBEC45F048C0EEFF49C0EDFF80
:106FA000D890C037C137BC2B100EBC5D0EE2C0516B
:106FB000BE15486EC151BF15496E4850491005E1D4
:106FC000BC2BD890C037C137EFD7100EBC5D02E3A1
:106FD0009D9C05D0BC51040DF328C26EC282F2A460
:106FE00035D0D59EF294F29A040E486E0701B7513F
:106FF000D1EC45F0EF50485C29E1080EB75D0AE29C
:107000000AEC46F004E0E846FE0B4806FCE1E81C0A
:10701000891616D0100EB75D0AE20AEC46F004E0BD
:10702000E846FE0B4806FCE1E81C8A1609D00AEC8B
:1070300046F004E0E846FE0B4806FCE1E81C8B162F
:107040000701B751D1EC45F0020EEF6E040EE15C82
:1070500002E2E16AE552E16EE552E5CFDAFFE7CF01
:10706000D9FFE552E5CFF4FFE5CFF3FFE5CFEAFF27
:10707000E5CFE9FFE550E5CFE0FFE5CFD8FF100011
:10708000EDEC46F0896A92680701BE6BBF6B8A6AB5
:1070900093688B6A94688C968C9495969594928E4E
:1070A000010EE36F0701F369F4690701B26BB16B7D
:1070B000B36BAD6BAC6BAE6BAA6BAB6BAF6BB06B0A
:1070C000B86BB96BBA6BBB6BBC6B76827680769C07
:1070D000769A76887696FA0E776EDF6ADFCF00F0C2
:1070E000100EE76E0018E8AE02D0E73402D0E75089
:1070F000005C0BE2DFCFE9FFEA6AE9BEEA68BBECBD
:1071000045F0EE6AED6ADF2AE9D70701DD6BDE6B39
:10711000DB6BDC6BDF6BE06BE16BE26BB56BB66B73
:10712000B76BDF6ADFCF00F0180EE76E0018E8AE2D
:1071300002D0E73402D0E750005C16E2DFCFE9FF6F
:10714000EA6AE9BEEA681FEC46F0EE6AED6ADFCF54
:10715000E9FFEA6AE9BEEA68290EE926010EEA2299
:10716000010EEF6EDF2ADED7D586D59AD59CF29434
:10717000F29AF1940F01498FBE0EC16ED08E7694B3
:10718000A386A59669EC27F0A6EC5DF0F28EF28C52
:107190007684E552E55210EF45F0EDEC46F0CBEC8D
:1071A00045F0030EDB6A040EDB6A34EC44F00701A1
:1071B000AE5100080AE256EC3EF00701AD2B030E7B
:1071C000AD5D01E1AD6BAE07F2D7B35100080AE245
:1071D00078EC3EF00701B22B030EB25D01E1B26B19
:1071E000B307F3D7200E0201E76E8019E8AE02D094
:1071F000E73402D0E750805D01E239D16550020BDF
:1072000001E035D1400EE66E400EE66E020EE66EEF
:107210003DEC5CF0FCEC46F0E76E030EE7CFDBFFE5
:10722000DB50000801E3E5D0040EDB6A030EDB50FF
:10723000F36E040EC1EC45F001E3DBD0040EDB502D
:10724000EA6A400FE96E020EEA22EFCFDFFF050186
:107250005D5132E10D0E41EC45F005E00A0E016E84
:10726000DF50015C29E1010E5D6F07017FEC45F005
:107270000D0EEF6EDD2B010EDB6ADD51F36E010E9C
:10728000C1EC45F014E216EC46F0E9BEEA68000EE7
:10729000E926030EEA22EF50E66E16EC46F0E9BE50
:1072A000EA68190EE926050E2BEC46F0E6D73CD924
:1072B0000701DD6BDE6B8DD01B0EDF5C09E15951E0
:1072C00007E1010E596F1B0E5A6F5B6B5C6B81D02F
:1072D00059050BE15B0EDF5C08E11B0E5A5D05E111
:1072E0005B5103E15B0E5B6F74D059054AE1410EBF
:1072F000DF5C47E11B0E5A5D44E15B0E5B5D41E1E3
:107300005A6B5B6B5C6B596B010EDB6ADBCFE9FF81
:10731000EA6AE9BEEA68000EE926030EEA22EF50A7
:107320000D0814E016EC46F0E9BEEA68190EE926ED
:10733000050EEA22EF50E66E16EC46F0E9BEEA686A
:10734000000EE926030E2BEC46F0E0D7010EDBCF52
:10735000DDF707017FEC45F0EF6A010E006EB30E1A
:1073600057EC46F0000EE66E030EE66EFE0E006E63
:10737000B20E63EC46F002E2E16AE552E16E0350C0
:1073800028D0080EDF5C0EE10701DD5100080AE29B
:10739000DD077FEC45F0EF6AFB0E006EB20E57EC96
:1073A00046F017D00D0EDF5C14E00A0EDF5C11E032
:1073B000200EDF5C0EE305015A6B5B6B5C6B596B57
:1073C00007017FEC45F0DFCFEFFF05015D6B0701A3
:1073D000DD2B0701DD51006E016A000E001806E189
:1073E000010E011803E1B487DD6BDE6B040EDB2AAE
:1073F0001DD70701B4513AE0B4A105D0F50E006ED7
:10740000B20E57EC46F00701B4A305D0D60E006EBD
:10741000B20E57EC46F00701B4A505D0BA0E006EC7
:10742000B20E57EC46F00701B4A705D09E0E006ED1
:10743000B20E57EC46F00701B4A905D07F0E006EDE
:10744000B20E57EC46F00701B4AD05D05E0E006EEB
:10745000B20E57EC46F0000E0701B41505E0450EDC
:10746000006EB20E57EC46F00701B46B37D8050E2C
:10747000E15C02E2E16AE552E16E10EF45F066EC94
:1074800046F0DBC7DFFFDF2A400E41EC45F001E1AB
:10749000DF6A0701DC51DF5C01E120D80701DB5125
:1074A000EA6A000FE96E020EEA22FD0EDBCFEFFF63
:1074B000DB2B400EDB5D01E1DB6BDC51DB5D01E1D1
:1074C000B485FD0EDBCF00F0016A00BE016800C08C
:1074D000F3FF01C0F4FFE55210EF45F066EC46F013
:1074E0000701DB51DC5D1DE00701905105E0C7ECB1
:1074F0005CF086EC47F0F8D70701DC51D880DB550B
:1075000007E2DC51DB5D58EC45F0DBC7DCF707D068
:10751000400ED880DC5558EC45F00701DC6BC7EC19
:107520005CF0E55210EF45F0EDEC46F0E652E65225
:10753000DE6ADD6A020EDB6A030EDB6A070120ECFD
:1075400045F032EC46F0020EF3CFDBFF07013AECD8
:1075500045F004E1010E011801E1DE6B020EDB5083
:10756000DE6EDD6A20EC45F02C0824E020EC45F0CE
:107570000D0820E020EC45F032EC46F0030EF3CF8E
:10758000DBFF07013AEC45F004E1010E011801E1CF
:10759000DE6B020EDBCF02F002C003F0026A030EC4
:1075A000DB5000010224006E000E0320016E00C0BB
:1075B000DEFFDD6E000EDFCF3AF0010EDBCF3BF0D9
:1075C000530E3A1802E1430E3B1801E1F7D1530E76
:1075D0003A1802E1510E3B1801E1EDD14D0E3A1877
:1075E00002E1580E3B1801E1E3D1530E3A1802E1D3
:1075F000450E3B1801E1D9D1430E3A1802E1410E84
:107600003B1801E1D0D14D0E3A1802E1510E3B1862
:1076100001E1C6D14D0E3A1802E1520E3B1801E1CC
:10762000BCD1320E3A1802E1530E3B1801E1B2D13F
:10763000450E3A1802E1530E3B1801E1A8D1430E62
:107640003A1802E1510E3B1801E19ED14B0E3A1857
:1076500002E1430E3B1801E194D14C0E3A1802E1CD
:10766000420E3B1801E18AD1440E3A1802E14E0E57
:107670003B1801E180D1490E3A1802E14E0E3B1849
:1076800001E176D1420E3A1802E1510E3B1801E1B8
:107690006CD14C0E3A1802E1510E3B1801E162D157
:1076A0004C0E3A1802E1530E3B1801E158D14E0E30
:1076B0003A1802E1510E3B1801E14ED14E0E3A1834
:1076C00002E1530E3B1801E144D1430E3A1802E1A6
:1076D000530E3B1801E13AD14D0E3A1802E1450E26
:1076E0003B1801E130D1500E3A1802E1510E3B181F
:1076F00001E126D1500E3A1802E1540E3B1801E187
:107700001CD1500E3A1802E1530E3B1801E112D180
:107710004D0E3A1802E1410E3B1801E108D14D0E21
:107720003A1802E1530E3B1801E1FED0470E3A1819
:1077300002E1500E3B1801E1F4D0430E3A1802E189
:10774000500E3B1801E1EAD0490E3A1802E1430E0F
:107750003B1801E1E0D0490E3A1802E1520E3B1805
:1077600001E1D6D0490E3A1802E1530E3B1801E16F
:10777000CCD0530E3A1802E1520E3B1801E1C2D0B0
:10778000530E3A1802E1530E3B1801E1B8D0530EE4
:107790003A1802E1420E3B1801E1AED0430E3A180E
:1077A00002E1420E3B1801E1A4D0430E3A1802E177
:1077B000520E3B1801E19AD04F0E3A1802E1420EE8
:1077C0003B1801E190D0570E3A1802E14D0E3B18DC
:1077D00001E187D0520E3A1802E14D0E3B1801E14B
:1077E0007ED0440E3A1802E1500E3B1801E175D0EC
:1077F0004F0E3A1802E1500E3B186DE0490E3A1850
:1078000002E1500E3B1865E0580E3A1802E1540EA2
:107810003B185CE0540E3A1801E13B5055E0410E34
:107820003A1801E13B504EE0560E3A1801E13B5048
:1078300047E0490E3A1801E13B5040E04F0E3A183C
:1078400001E13B5039E0550E3A1802E1430E3B1876
:1078500031E0580E3A1802E1430E3B1828E0430E7F
:107860003A1801E13B5021E0520E3A1801E13B5039
:107870001AE0580E3A1802E1520E3B1811E0030EBE
:10788000DB5001E09ED0020EDBEC45F0DBEC45F076
:10789000220E006EB20E8FEC46F001E3A1D09ED016
:1078A000AAEC40F09FD0C3D89DD029D99BD0ACEC96
:1078B00040F098D0C0D896D0C5D994D0F7D992D0FE
:1078C00012DA90D015DA8ED0F1D88CD0A8EC40F036
:1078D00089D036DB87D0A7DB85D09DDA83D07CDAF0
:1078E00081D068DA7FD01EEC41F07CD0AEEC40F065
:1078F00079D01CEC41F076D020EC41F073D022EC32
:1079000041F070D024EC41F06DD026EC41F06AD00B
:1079100028EC41F067D02AEC41F064D02CEC41F027
:1079200061D086EC41F05ED0BCEC2BF05BD004EC77
:1079300029F058D03DEC2FF055D01EEC2FF052D04E
:107940000BEC2FF04FD0B7EC2FF04CD03DEC28F0E3
:1079500049D038EC30F046D056EC30F043D068ECEB
:1079600030F040D075EC30F03DD087EC30F03AD0BC
:107970001AEC30F037D02BEC30F034D0BBEC41F0C7
:1079800031D0C3EC41F02ED09BEC30F02BD0AFECDB
:1079900030F028D01DEC5EF025D044EC31F022D040
:1079A00045EC31F01FD03AD91DD083EC2EF01AD01F
:1079B00057EC2CF017D019EC32F014D04CEC32F01C
:1079C00011D0A0EC46F0A0EC46F0FA0E006EB10E1D
:1079D00001EC45F0036E0B0EE15C02E2E16AE55258
:1079E000E16E0350070120EC45F00D080DE0B451A5
:1079F0000BE1520E006E016ADF50001803E1DE5207
:107A0000DD50011801E0B48FDDC7DEF7040EE15C44
:107A100002E2E16AE552E16E10EF45F00701E35141
:107A200005E0320E006EC70E57EC46F0120040EC37
:107A300038F00EEF3DF066EC46F0DEEC46F01BEC65
:107A400045F0020EE3EC46F02FE1DF0414E1D950DB
:107A5000010FF1EC45F00AE0010E006E016ADB5007
:107A6000001808E1020EDB50011804E1010EDBCF23
:107A7000E3F701D0B48D020E41EC45F014E1D9508A
:107A8000010FF1EC45F00AE0010E006E016ADB50D7
:107A9000001808E1020EDB50011804E1010EDBCFF3
:107AA000BFFE01D0B48DBADF69EF46F00AEC45F0B5
:107AB000CBEC45F0E66AA80EE66E070EE66E04EC27
:107AC00047F01BE1020EDB500CE1A851A91103E1C4
:107AD000AA6BAB6B11D07684A8C7AAF7A9C7ABF77E
:107AE0000BD0A851A91103E1AF6BB06B05D0768420
:107AF000A8C7AFF7A9C7B0F791DF69EF46F0EDEC83
:107B000046F0E652DEEC46F013EC47F0020F13ECC1
:107B100047F0030F13EC47F0040F5AEC46F00FE167
:107B2000DF50926E010EDB50936E020EDB50946EAE
:107B3000030EDB50956E040EDB50966E6FDF050E64
:107B4000E15C02E2E16AE552E16E10EF45F00AEC19
:107B500045F0FD0EDB50100805E2100EF36EFD0E31
:107B6000F3CFDBFFFC0EDB502AE0FD0EDB50F6EC22
:107B700063F0F3500701BE13F450BF13080EF36E09
:107B8000FD0EC1EC45F00DE2010EF36EFD0EDB5073
:107B900003E036EC45F0FDE1F350F31C0F0148170C
:107BA0003BD0FD0EDB500C0837E339EC46F003E028
:107BB0001BEC46F0FDE1E81C0F0149172DD0FD0E2E
:107BC000DB50F6EC63F0F3CF00F0F4CF01F0001ED1
:107BD000011E00500701BE170150BF17080EF36EBB
:107BE000FD0EC1EC45F00CE2010EF36EFD0EDB5014
:107BF00003E036EC45F0FDE1F3500F0148130CD0E3
:107C0000FD0EDB500C0808E339EC46F003E01BECFA
:107C100046F0FDE10F01491310EF45F00AEC45F085
:107C2000DEEC46F05AEC46F009E1010EDBCFE6FF50
:107C3000DFCFE6FF8CDFE552E552F0DEE552E5529C
:107C400010EF45F00AEC45F029EC45F0010EFEEC92
:107C500044F066EC45F026E1010EDB5002E1DF5016
:107C6000896E70EC46F01EE1010EDB5002E1DF5040
:107C70008A6E70EC46F016E1010EDB5002E1DF5037
:107C80008B6E70EC46F00EE1010EDB5002E1DF502E
:107C90008C6E70EC46F006E1010EDB5002E1DF5025
:107CA0008D6EBCDEE552E55210EF45F08450E66E75
:107CB000E66A8350E66EE66A8250E66EE66A8150B6
:107CC000E66EE66A8050E66EE66ADD0E006EB10E84
:107CD00001EC45F0036E0D0EE15C02E2E16AE55253
:107CE000E16E035012003A0E006EC70E57EF46F0D9
:107CF000EDEC46F0E652DF6A010EF36EDB6E020E2B
:107D0000DB6ADB0E006EB10E57EC46F09DBCFED771
:107D1000DF6ADFCF00F0100EE76E0018E8AE02D089
:107D2000E73402D0E750005C3EE2010EDB50070171
:107D3000BE150001006E020EDB500701BF150001E9
:107D4000016E005001101EE0DFCFE9FFEA6AE9BED4
:107D5000EA68BBEC45F0EECFE6FFEFCFE6FFDFCF02
:107D600000F0016A00BE0168C9EC46F0D00E026E58
:107D7000B10EDFEC45F0070EE15C02E2E16AE5528C
:107D8000E16E0550010EDBCF00F0020EDBCF01F0FB
:107D9000D89000360136010E00C0DBFF020E01C094
:107DA000DBFFDF2AB6D7370E006EC70E57EC46F062
:107DB00069EF46F066EC46F029EC45F004EC47F03C
:107DC00009E101EC46F005E2CEEC46F0020EDBCF15
:107DD000EFFF24DE69EF46F066EC46F029EC45F053
:107DE000030EE3EC46F015E101EC46F005E2CEECC3
:107DF00046F0020EEFCFDBFF020EDBEC45F0C60EC5
:107E0000006EB10E63EC46F002E2E16AE552E16E0B
:107E1000035069EF46F017EC47F001E08FD0020EF7
:107E2000DB50010801E287D0010EDB50070801E2B8
:107E300082D0410E41EC45F016E1020EDB500AE122
:107E400045EC45F003E036EC45F0FDE1F350F31C62
:107E5000921673D045EC45F003E036EC45F0FDE1B9
:107E6000F35092126AD0420E41EC45F016E1020E38
:107E7000DB500AE145EC45F003E036EC45F0FDE16E
:107E8000F350F31C931659D045EC45F003E036EC63
:107E900045F0FDE1F350931250D0430E41EC45F014
:107EA00016E1020EDB500AE145EC45F003E036EC4A
:107EB00045F0FDE1F350F31C94163FD045EC45F03E
:107EC00003E036EC45F0FDE1F350941236D0440E59
:107ED00041EC45F016E1020EDB500AE145EC45F0BD
:107EE00003E036EC45F0FDE1F350F31C951625D088
:107EF00045EC45F003E036EC45F0FDE1F35095121A
:107F00001CD0450E41EC45F016E1020EDB500AE1B3
:107F100045EC45F003E036EC45F0FDE1F350F31C91
:107F200096160BD045EC45F003E036EC45F0FDE14C
:107F3000F350961202D0B48D01D070DD69EF46F097
:107F40000AEC45F0CBEC45F00DEC47F0050E53EC98
:107F500046F0010F5AEC46F064E1010EDB500708D1
:107F60004CE3410E41EC45F00AE190EC45F003E0B2
:107F70001BEC46F0FDE1E8407F0B801437D0420E49
:107F800041EC45F00AE190EC45F003E01BEC46F0D3
:107F9000FDE1E8407F0B811429D0430E41EC45F010
:107FA0000AE190EC45F003E01BEC46F0FDE1E8400F
:107FB0007F0B82141BD0440E41EC45F00AE190EC9B
:107FC00045F003E01BEC46F0FDE1E8407F0B831435
:107FD0000DD0450E41EC45F010E190EC45F003E08A
:107FE0001BEC46F0FDE1E8407F0B8414E76E020EC7
:107FF000E7CFDBFFDB5008E002D0B48D12D0010EDA
:10800000F36E020EF3CFDBFF020EDBEC45F0BD0E8C
:10801000006EB10E63EC46F002E2E16AE552E16EF9
:10802000035069EF46F017EC47F001E08FD0020EE5
:10803000DB50010801E287D0010EDB50070801E2A6
:1080400082D0410E41EC45F016E1020EDB500AE110
:1080500045EC45F003E036EC45F0FDE1F350F31C50
:10806000891673D045EC45F003E036EC45F0FDE1B0
:10807000F35089126AD0420E41EC45F016E1020E2F
:10808000DB500AE145EC45F003E036EC45F0FDE15C
:10809000F350F31C8A1659D045EC45F003E036EC5A
:1080A00045F0FDE1F3508A1250D0430E41EC45F00B
:1080B00016E1020EDB500AE145EC45F003E036EC38
:1080C00045F0FDE1F350F31C8B163FD045EC45F035
:1080D00003E036EC45F0FDE1F3508B1236D0440E50
:1080E00041EC45F016E1020EDB500AE145EC45F0AB
:1080F00003E036EC45F0FDE1F350F31C8C1625D07F
:1081000045EC45F003E036EC45F0FDE1F3508C1210
:108110001CD0450E41EC45F016E1020EDB500AE1A1
:1081200045EC45F003E036EC45F0FDE1F350F31C7F
:108130008D160BD045EC45F003E036EC45F0FDE143
:10814000F3508D1202D0B48D01D068DC69EF46F097
:108150000EEF3DF00EEF3DF00EEF3DF0EDEC46F092
:10816000D8EC46F087EC46F060E1D950020FD3EC32
:1081700046F0720ED880EE542E0EED543BE3D950EB
:10818000020FF1EC45F01FE003680468056A2D0E4C
:10819000E76E020EDBCF06F0030EDBCF07F0E750F1
:1081A0000626000E0722086A0650035C006E075080
:1081B0000458016E08500558026E020E00C0DBFF25
:1081C000030E01C0DBFF010EDB50070813E3410E75
:1081D00041EC45F002E1DF6A0FD0420E41EC45F080
:1081E00002E1080E05D0430E41EC45F003E1100E0C
:1081F000DF6E02D0B48D19D0010EDB50DF24E96EA2
:10820000EA6A1FEC46F040EC46F0010EDB50DF243A
:10821000D1EC45F0EF0407E1010EDB50DF24D1EC97
:1082200045F0020EEF6E0EEC3DF0040EE15C02E252
:10823000E16AE552E16EF4D30EEF3DF00EEF3DF052
:108240000EEF3DF00EEF3DF00EEF3DF00EEF3DF086
:108250000EEF3DF00EEF3DF0DDDB070EE12402E313
:10826000E168E652E16E0DEC47F0030E53EC46F088
:1082700087EC46F044E1DECF01F5DDCF02F5020EDA
:10828000DBCF09F5030EDBCF0AF5040EDB6A030E24
:10829000F36E040EC1EC45F030E26DEC45F0030ED8
:1082A000ADDBE76E050EE7CFDBFF010EE66ED950C2
:1082B00009EC47F0A3DBE76E060EE7CFDBFF070113
:1082C000B4511DE1050EDB5018E1060EDB5015E13F
:1082D00025EC46F0010EE926050EEA22DECFEEFF80
:1082E000DDCFEDFF25EC46F0090EE926050EEA226A
:1082F00040EC46F0040EDB2ACAD70EEC3DF0070E28
:10830000E15C02E2E16AE552E16E8AD366EC46F096
:108310000DEC47F0010EE3EC46F00DE1DF5007E015
:10832000F00E9314936E0501010E006F02D005014B
:10833000006B0EEC3DF0E55273D3D9CFE6FFDACFF8
:10834000E6FFE1CFD9FFE2CFDAFFE652DF6AFF0EA8
:10835000DF5C0AE2E868E85005E0E80600D000D0FB
:1083600000D0F9D7DF2AF3D7E552E552E5CFDAFF9F
:10837000E7CFD9FF1200F29EF29C6592656ADDDFBD
:108380000FEF00F0120046DB100EE12402E3E1687B
:10839000E652E16EE66AD950010F4DDBE66AA5ECC4
:1083A00046F00DEC47F0010E53EC46F0040F43DBB2
:1083B000020E53EC46F009EC47F053EC46F00A0F7E
:1083C0003ADB060E53EC46F0060F35DB070E53EC96
:1083D00046F00E0F30DB040E53EC46F00F0F2BDB94
:1083E000050E0CDB010EDBCF00F0016A00BE016858
:1083F000C9EC46F0B10E026EB10EE1DB050EE15C98
:1084000002E2E16AE552E16E0550DFCFE6FFE66A7F
:10841000A50E006EB10E63EC46F002E2E16AE55291
:10842000E16E0350040EDBCFE6FF050EDBCFE6FF67
:10843000990E006EB10E63EC46F002E2E16AE5527D
:10844000E16E0350020EDBCFE6FF030EDBCFE6FF4B
:108450008D0E006EB10E63EC46F002E2E16AE55269
:10846000E16E0350D9500A0F6FDB800E006EB10E23
:108470008FEC46F002E2E16AE552E16E0350D9501A
:10848000060F62DB730E006EB10E8FEC46F002E257
:10849000E16AE552E16E03500E0E8DDB670E006E51
:1084A000B10E63EC46F002E2E16AE552E16E035080
:1084B0000F0E81DB5B0E006EB10E63EC46F002E244
:1084C000E16AE552E16E03500EEC3DF0100EE15C06
:1084D00002E2E16AE552E16EA3D29CDA090EE124E0
:1084E00002E3E168E652E16E080EDB6A0D0E006EF3
:1084F0000701A6DA005C05E1FA0EDB5027E1B4893A
:1085000025D09EDA2C0813E0FA0EDB500EE198DA43
:10851000E66EE66A340E006EB10ED5DB02E2E16A69
:10852000E552E16E03500701B48B020E25D1A2DAA9
:1085300004E1010E011801E1DE6B0D0E006E80DA20
:10854000005C06E1FA0EDB5001E1B489030E14D1A0
:108550002D0E006E75DA005C20E1040E4DDB1DE08F
:10856000050E026EFD0EDB50025C17E0FD0EDB0413
:1085700001E1C8D0030E0ADB01E1C4D0070E3CDBE9
:1085800001E1C0D0010EF36E080EF3CFDBFF72DA0B
:1085900004E1010E011801E1DE6B040EF7DA0AE0D6
:1085A000050E2ADB07E00A0EE66E95DBEED8FCEC42
:1085B00046F036D0DE519DDBEFCF00F0000E00C05C
:1085C000DFFF010EDB6A020EDB6A030EDB6A050EBB
:1085D000DDDA1FE1000EDFCFE6FF010EDBCFE6FFA5
:1085E0004FEC63F0E552E552F3CF00F0F4CF01F029
:1085F000026A036A01AE02D00268036800C0DFFFAE
:10860000010E01C0DBFF020E02C0DBFF030E03C040
:10861000DBFF07012FDA04E1010E011801E1DE6B37
:10862000080EDB5042E0FD0EDB5007E110EC47F096
:10863000800E38DA000EEE5412E3020EA7DA06E1DD
:10864000EFDB000EEE54800E2DDA09E3060ED4DACD
:1086500008E1E6DB000E26DA800EEE5402E20701A6
:1086600051D0F2D97BDA080EDB5054E0040EDBCF98
:1086700038F0050EDBCF39F0060EDBCF3AF0070EEF
:10868000DBCF3BF03D683E683F68406817EC63F025
:10869000040E34C0DBFF050E35C0DBFF060E36C00E
:1086A000DBFF070E37C0DBFF35D0FD0EDB5006E1E8
:1086B000B7DB7F0EEE54000EF5D923E3FD0EDB048D
:1086C00004E11DDB000EEED91CE3020E5FDA04E1CB
:1086D00016DB7F0EE7D915E3030E8EDA04E10FDB1C
:1086E000FF0EE0D90EE3060E026EFD0EDB50025CBB
:1086F0000CE105DBFF0EEE54FF0EEE547F0EEE5440
:1087000004E20701B48D010E37D0070E3FDA02E014
:108710009BD924DAFD0EDB50070A21E0010A17E09D
:10872000050A11E0010A0FE0030A08E0050A06E065
:10873000010A04E0050A02E0040E1ED0E3D9040E8B
:10874000DBCFEFFF18D006DBDBCFEDFF14D002DB71
:10875000DBCFEEFF060EDBCFEEFF070E0AD0D2D93D
:10876000DFCFEEFF010EDBCFEEFF020EDBCFEEFF21
:10877000030EDBCFEEFF000E006E090EE15C02E29D
:10878000E16AE552E16E00504BD127DB2EDAEE6A4A
:10879000EE6AEE6AEE6A010EDB6AFB0EDB50F36EE8
:1087A000010EEFD94FE20701DE51A3DAEFCFDFFF71
:1087B000300EDF5C42E3DF5039083FE316DAEECFDC
:1087C00000F0EECF01F0EECF02F0EFCF03F00A0E93
:1087D0003D6E3E6A3F6A406A00C038F001C039F021
:1087E00002C03AF003C03BF017EC63F034C000F075
:1087F00035C001F036C002F037C003F0300EDF5C48
:10880000046E056A066A076AE850002605500122D0
:108810000650022207500322E8D900C0EEFF01C033
:10882000EEFF02C0EEFF03C0EEFF070123D907E110
:10883000010E011804E1DE6B02D0000E04D0010E1F
:10884000DB2AABD7010EE552E552EAD00701AE5163
:10885000E66EE66A280E006EB10E35DA02E2E16AD3
:10886000E552E16E035012000201805108E0010E52
:10887000006E6550020B01E0010E005C17E1D0D9DB
:108880000BE16151621111E18C86A00E616F0F0E38
:10889000626F010E636F12006151621152E18C969A
:1088A000A00E616F0F0E626F636B1200800509E00E
:1088B000020E805D06E0040E805D03E0100E805D18
:1088C00017E1AED90BE16151621111E18C86200EE6
:1088D000616F4E0E626F010E636F12006151621183
:1088E00030E18C96200E616F4E0E626F636B12004A
:1088F000200E805D26E194D907E16151621121E1EA
:108900008C86CCD9010E15D0630507E16151621147
:1089100018E18C96C3D9020E0CD0020E635D0BE1F8
:10892000615162110EE18C86A00E616F860E626F3E
:10893000030E636F12006151621103E18C96AED990
:10894000636B120067D8A3D9E8AE02D0003403D01D
:10895000E750D880005423E3FC0EDB5010E0CAD867
:10896000E9BEEA6896D804E0E846FE0B0106FCE1A1
:10897000006EC0D8E9BEEA6833DAEF1210D0BAD878
:10898000E9BEEA6886D804E0E846FE0B0106FCE191
:10899000E81C006EAFD8E9BEEA6822DAEF1640D0D4
:1089A00039D875D9E8AE02D0003403D0E750D8806A
:1089B000005423E3FC0EDB5011E19CD8E9BEEA68C9
:1089C00068D804E0E846FE0B0106FCE1E81C006EF6
:1089D00091D8E9BEEA680ADAEF160FD08BD8E9BE63
:1089E000EA6857D804E0E846FE0B0106FCE1006E99
:1089F00081D8E9BEEA68FAD9EF1212D0E66EA5EF87
:108A000046F0016E026A00C0E6FFE66E02C0E6FFB5
:108A100041EF62F060D9E1CFD9FFE2CFDAFF120077
:108A2000E552E5CFDAFFE7CFD9FF1200A951E96E91
:108A3000EA6A83EF46F0E66E000EDA20E66E120078
:108A4000DE5157D9EF501200D9CFE9FFDACFEAFF54
:108A50001200E652E6520DEF47F0EA22EECF48F060
:108A6000EFCF49F012009AD9010E1200D890F336D8
:108A7000E8061200DE2BDE51006E016A000E0018BF
:108A80001200006EDF50005C1200010EF36EDB502E
:108A90001200C80EE926050EEA22EF50016E010E03
:108AA00001521200EE54000EEE54000EEE5412006D
:108AB000DF6EDFCFE6FFDC51016A000F006E020EB1
:108AC000012267D980EC5CF0FCEF46F0E76E010E06
:108AD000E7CFDBFF0701B4511200010EE66E6BEF2A
:108AE00046F0EA22EECF4AF0EFCF4BF012000BD95E
:108AF000E8061200FD0EDBCFE9FFEA6A1200DD5145
:108B000079EF46F0FB0EDBCFE9FFFC0EDBCFEAFF8F
:108B10001200EA22EE50EFCFEAFFE96E0050120099
:108B2000010EDB28006E010E00521200A951EA6A04
:108B3000310FE96E0E0EEA22EF500E01EA6AAC2503
:108B4000E96EAD51EA2212002ED9EECFE6FFEECF4C
:108B5000E6FFEECFE6FFEFCFE6FF1200040EEECF0A
:108B6000DBFF050EEECFDBFF060EEECFDBFF070EC1
:108B7000EECFDBFF1200C7D8000EE926010EEA2275
:108B80001200DBCFF4FFF350F45C1200006EFD0E18
:108B9000DB50005C1200E652E652E652020EDB6A3F
:108BA0001200EA6A290FE96E010EEA221200036E32
:108BB000050EE15C1200DBCFE6FFE66A1200036EF1
:108BC000046A02C0E6FFE66E04C0E6FF41EC62F014
:108BD000056E1200020EDBCF48F0030EDBCF49F02A
:108BE0001200E1D8EE50ED101200FC0EDBCFE9FFD1
:108BF000FD0EDBCFEAFF1200016EFD0EDB50015CC3
:108C00001200DECF00F0DDCF01F0000E005C100E90
:108C100001581200070EB715486E010E4852120097
:108C200005016107000E625B63511200010EDBCF8C
:108C3000E9FFEA6A1200E846FE0B0006120063D85C
:108C4000410EE926010EEA221200040EDB28E96E2D
:108C5000EA6A83EF46F0EA22E552E750EF6E010E32
:108C6000DB2A1200E66EE66A4FEC63F0E552E5524D
:108C70001200FD0EDB50F80F006E010E00521200C4
:108C8000020EDBCFEEFF030EDBCFEDFF1200FD0E79
:108C9000DBCF00F0190EE76E00181200100E616FA6
:108CA000270E626F1200AADEE66AD9501200A9DE12
:108CB000FCEF46F0C0DE010EE3EF46F0B7DE010E3A
:108CC000E9260E0E12009DDED7EF45F0A3DEE65238
:108CD000120092D8A5D6D9CFE6FFDACFE6FF120070
:108CE000FCDE8CDE66EF45F0A1DE790EE9260E0E85
:108CF0001200EA6A000FE96E030EEA22120090D811
:108D0000FF0EEE541200D890E936EA36120081D8F0
:108D1000E3EF46F08BDE490EE9260E0E120071DEFF
:108D2000036E070EE15C1200110EE926050E95DEBA
:108D300033EF45F0D6DE48504A5C49504B5812009C
:108D4000030E39DF020EDBEF45F06DEC42F054D834
:108D5000E5521200D7DE040EDBCFEEFF050E120047
:108D6000C0DE4A5048181200110EE926050EEA220C
:108D700012006ADEEE50ED10120066DE010EEE18F3
:108D8000120062DE020EEE1812005EDE030EEE1816
:108D9000120000C0E6FF01C0E6FF1200DECFE9FFCF
:108DA000DDCFEAFF1200E96E000EDA20EA6E120053
:108DB00050DE050E78DF010F13EF47F04ADE010E9B
:108DC00072DF010F12001ADE0701B45112008CDFAE
:108DD00044DE74DFEA224850120078DFE6521200C7
:108DE00092DF960EE926050E89EF45F08CDF640EC2
:108DF000E926050E89EF45F0E552E552E5521200ED
:108E000089DF2BDE5EEF46F0030E4DDF020F5AEFD7
:108E100046F0020F10DE030E1200E66A6BEF46F01A
:108E200013DED880120007DE010E53EF46F04EDF4E
:088E3000BFDF020F5AEF46F00C
:088E3800B3EC4CF0A098636A52
:108E4000626A0F01266B8AEC4DF002E2E16AE5529C
:108E5000E16E00500F0147EC4DF0DF6ADF50006E0D
:108E6000016A0C0E005C000E015810E2DF50040D88
:108E7000F3CFE9FFF4CFEAFF000EE926040EEA2261
:108E8000EE6AEE6AEE6AEE6ADF2AE8D7658C0F01B9
:108E9000386B6598659C62A607D062960201976B55
:108EA0009C6B9D6B9E6BF7D70201010EB06FB16F8B
:108EB000B26BB36BA46BDF6A030EDF5C11E2EA6A8C
:108EC000DF34B7EC4DF0EA22EE6AED6AEA6ADF348D
:108ED000BEEC4DF0EA22EE6AED6AF1EC4CF0ECD714
:108EE0000201080E8D6F040E8E6F0F01160E266F95
:108EF0000401300E026F040E036F400E016F840EEA
:108F0000006F0201816B806BB6EF4CF0B3EC4CF05C
:108F100082BE06D0656A0F01366B0201806B7CD081
:108F2000020180510CE1656A0F01366B47EC4DF090
:108F300065B602D06586FCD70201010E806F800500
:108F40000AE165BA08D0626A0F01366B368136894C
:108F50000201020E806F6250040B06E00F013651D1
:108F6000040B02E062943EDB65B256D06250010B06
:108F700009E00F013651010B05E05EDF0201040E2E
:108F8000806F62906250100B06E00F013651100B9B
:108F900002E018DB629862AC15D00F0136AD0AD042
:108FA0004EEC4DF0730EBDEC4CF002E2E16AE5527E
:108FB000E16E0050629C0201AE5101E0AE07AE517D
:108FC00001E1F3D86250200B05E00F013651200B70
:108FD00001E0E7DA6250020B14E00F013651020B98
:108FE00010E04EEC4DF0E6687F0EE66E9BEC5FF015
:108FF000006E060EE15C02E2E16AE552E16E0050AD
:10900000636A040E0201E76E8019E8AE02D0E7340D
:1090100002D0E750805D02E2A19834D00F0136A75C
:1090200030D0DF6A040EDF5C2CE262A62AD064CF67
:10903000A5F20201A551780BE842E842E842A66F8A
:109040006296A5B504D0A651C5EC4DF003D0A6514B
:10905000CAEC4DF0EA22EF70A65102E1D5DA0FD04A
:10906000000EE66EE66AA50EE66E020EE66E720E63
:10907000BDEC4CF002E2E16AE552E16E0050DF2AFD
:10908000D1D7A198B6EF4CF0B4EC4DF0FC0EDBA4B8
:1090900003D0E66A2FEC4DF0FC0EDBA204D0010EEB
:1090A000E66E2FEC4DF0FD0EDB50016A260F006ED0
:1090B0000F0E29EC4DF0C5EC4CF0FC0EDBCFEFFFB2
:1090C000E552B6EF4CF0B4EC4DF0FC0EDB5003E093
:1090D000B8EC4CF002D0E2EC4CF015EC4DF0D9CFEE
:1090E000E9FFDACFEAFFEE50ED1003E1F36AF46A2C
:1090F00028D0C5EC4CF0D9EC4DF0FA0EDBCFEEFFEA
:10910000FB0EDBCFEDFFC5EC4CF0EE52F90EDBCFE2
:10911000EFFF400ECFEC4DF0880EDEEC4DF0FC0E74
:10912000DB5003E0B8EC4CF002D0E2EC4CF0EA2269
:10913000EF74DECF00F0DDCF01F000C0F3FF01C01F
:10914000F4FFE552B6EF4CF0B4EC4DF0FD0EDB5001
:1091500003E193EC4DF009D0E7EC4CF068EC4DF0F6
:10916000E7EC4CF0010F68EC4DF0E552B6EF4CF037
:109170009AEC4DF065A817D0ADEC4DF0400EEE1610
:10918000EE6AEE6AEE6AADEC4DF0EE7CB8EC4CF0B7
:10919000EA22EF74400E006EADEC4DF00050EF1679
:1091A000ADEC4DF0EF7C84EF4DF00201B05123E1C6
:1091B000010EB06FB1511FE1010EB16F020E945D4F
:1091C00007E1E8DBEE52EF6AE5DBC80EEF6E120056
:1091D000940511E1A76BD7EC4CF0EE52400EEF6E08
:1091E000E6DB74EC4DF0E3DB840EEF6E010EA76F4F
:1091F000B6DB800EEF6E12000201B26BB36B020E93
:10920000945D06E1D3EC4DF0D7DB63EC4DF010D06C
:1092100098510401365D020199510401375904E265
:1092200036C498F237C499F25CD8B4DBC5DBB2DB44
:10923000C80EEF6E1200B4EC4DF0000EDE6E040EA0
:10924000DD6EC5DB040DF4CF01F0D9CFE9FFDACF35
:10925000EAFFF350EE260150ED2297DBEF9EFC0E65
:10926000DB5002E1AFDB01D083DBEA22DECFEEFF91
:10927000DDCFEDFF8ADBEF9C88DB040EE926000ED4
:10928000EA22EF8CE55272D36598020197BF0DD0A8
:109290009CAF09D0020E946FB35101E1ADDF020122
:1092A000B16BB06B120093EF4DF0040130AF0DD0F5
:1092B0000201010E946FB25101E19EDF0201B16B18
:1092C000B06BAF510DE1D5EF48F00201020E946F83
:1092D00046DB840EEF6EB16BB06BAF5101E165DF21
:1092E000120041DB400EDF6E0201985D000E9959BD
:1092F0000AE298C2DFFF935102E1010E03D0930509
:1093000002E1020E936FDF50016AE850985D986F9A
:1093100001509959996F3EDBEE52DFCFEFFF380EC7
:10932000A16F040EA26F97B10DD0DF5017E095C268
:10933000F6FF96C2F7FF952B000E96230800F55016
:1093400067DBF3D7DF500AE095C2E9FF96C2EAFF78
:10935000952B000E9623EF505BDBF4D707D3B4ECCC
:109360004DF025DBEE52EFCFDFFFDFCF00F00050F6
:1093700002019D5D000E9E5902E29DC2DFFFDF509B
:10938000006E016AE8509D5D9D6F01509E599E6F71
:10939000010EDB6ADF50F36E010EDBCFF4FFF350FA
:1093A000F45C16E2010EDB50EA6A380FE96E040E37
:1093B000EA22EF50E66E9AC2E9FF9BC2EAFF9A2BBF
:1093C000000E9B23E552E750EF6E010EDB2AE2D739
:1093D000000ED8809D55000E9E550DE2E4DBECDAC0
:1093E000E6DAEF50400B03E16EDBC80E02D06BDB18
:1093F000880EEF6E12D0B3DA840EEF6E9F51A0117B
:1094000007E005D0A0C2FAFF02019F51F96EFADF12
:1094100002019C9FAF5101E1C8DEE552A7D2A3DA59
:109420000201978F77DB02E2E16AE552E16E0050BC
:10943000300EE66EE66AE66A000EE66E040EDBDAD1
:1094400002E2E16AE552E16E0050658CDF6A030ECC
:10945000DF5C02E2C6DAFBD7010EE66EE66AE66A78
:10946000820EE66E020EC7DA02E2E16AE552E16EB2
:109470000050659C0201080E8D6F040E8E6F000E69
:10948000836F040E846F83C285F2866F32C481F2CB
:10949000815102E1100E10D0010EE66EE66A810ED7
:1094A000E66E020EE66E010E68DA02E2E16AE5524D
:1094B000E16E00500201200E806F58D2800E040130
:1094C000305D38E10201C00E976F04013351030A89
:1094D0001AE0010A09E0030A2BE102011A0E956F56
:1094E000C50E966F120E1ED0E7DAA10EF626C50E37
:1094F000BEDA020E0201D9DAF5CF98F2030ED5DA00
:10950000F5CF99F21200030E325D0FE2D5DAA30E09
:10951000F626C50EACDA95C2F6FF96C2F7FF080034
:10952000F5500201986F996B12000201976B1200BF
:109530000201976B120018DB0401386B396B305154
:109540001F0B020A11E0030A0CE0010A1EE10201EE
:10955000978F040138810201A30517E104013883C4
:1095600014D00201978F11D00201978F040134BFEC
:1095700002D0E9DA01D0ECDA58DAF2DA06E005DAFC
:10958000EF50040B02E0010E386F020197AF07D0D5
:10959000380E956F040E966F9781020E986FE55204
:1095A000E5D10F0126A10CD002DAEF50800807E1C7
:1095B000F1D9EF50840803E1FAD98C0EEF6E2691B1
:1095C000629A12000F013685629865820201010ECF
:1095D000A46F31DA750ED1D902E2E16AE552E16E8B
:1095E000005012000201A46B26DA740EC6D902E202
:1095F000E16AE552E16E005065920F01369562A472
:1096000002D06294FCD71200AED902012D0EAE6FCB
:10961000FD0EA51539E17E0EA515E8407F0B040D62
:10962000F3CF83F2F4CF84F2000E8327040E842359
:1096300083C285F284C286F28575B9D9EF503C0B9E
:10964000E842E8420D081EE1DF6A080EDF5C16E220
:10965000AED9020EE926000ED5D9EF50E66EDF50E6
:10966000EA6A300FE96E040EEA22E552E750EF6E27
:109670009ED99FDAEE2AEF22DF2AE7D798D934DA8B
:1096800009D807D027D805D0FD0EA515040801E19B
:1096900030D86CD10201936BAF6BB26BB36BA76B1D
:1096A000946B78D9EF9E8D7575D9EF9E8D750BDA19
:1096B000EF9E976B986B996B9C6B9D6B9E6B55D8CF
:1096C000BAD9030E5AD902E2E16AE552E16E0050BE
:1096D00044EF49F0020E0201945D02E1AFEF49F060
:1096E000946BA75104E13BD98C0EEF6E1200A76B6F
:1096F000120039D94FD9EF50400B01E0010EDF6E57
:1097000002018D75080E805D0BE132C438FF0F0138
:10971000385103E00201100E02D00201040E806FE6
:10972000940513E137D948D9DCDD020E0201935DBF
:1097300003E130D9840E07D0DF5003E12BD9C80EE6
:1097400002D028D9880EEF6E0FD09CAF0CD09F515D
:10975000A01107E005D0A0C2FAFF02019F51F96EE7
:10976000FADF02019C9F946B01D104013051600B20
:10977000E842E842E842E842E842000901E012001B
:1097800031510C0A4AE00B0A3FE00C0A31E0010AB1
:1097900022E00B0A1EE0020A1CE0030A18E0080A95
:1097A00010E0010A0CE00F0A08E0030A01E01200D1
:1097B0000201978F080E806F12005EEF4AF00FEFE4
:1097C0004AF00201810E956F020E966F0CD09BEF4E
:1097D0004AF00EEF4CF034510201956F966B820EF9
:1097E0009527020E96239781010E986F978F12008E
:1097F0000201978F04013451EA6A820FE96E020E6A
:10980000EA2232C4EFFF120016D9020EB6D802E2E5
:10981000E16AE552E16E005012001200A5D9E6524D
:10982000E652E6520401320510E130511F0B0009E7
:109830000CE10201978F030E0401315D04E1020186
:10984000010EA36F02D00201A36B0401325101E0AB
:109850007FD030511F0B020801E07AD034510F0B3A
:10986000000901E175D034510F0B020871E3200E9D
:109870000201805D6DE1978F040134BF04D063D98C
:10988000D4D8DFD803D064D9D0D8DFD8EA22020EEA
:10989000EFCFDBFFF4D8010B02E1DF9401D0DF84CE
:1098A00034BF02D050D901D053D9EA22DECFEEFF27
:1098B000DDCFEDFF030E315D0CE152D907E034BF7F
:1098C00002D0BFD801D0C1D8EA22EF82840E76D967
:1098D0003FD0DF7445D90BE058D8EF9E56D8EF8CB7
:1098E00009D902E2E16AE552E16E005002D04DD89A
:1098F000EF8CDF74C4D8020B02E132D912E004010C
:1099000034BF02D09ED801D0A0D8EA22EF923B0EFD
:10991000006E45D9EFD802E2E16AE552E16E0050EF
:1099200002D03B0E3CD9040134510F0B016A260FC3
:10993000006E0F0E0122030E00C0DBFF040E01C0FB
:10994000DBFF030EDBCFE9FF040EDBCFEAFFEF9076
:10995000050EE15C02E2E16AE552E16ED5D023D961
:10996000C3D863EF4DF0E6D8E6521200E552CCD0F2
:10997000FD0EEA6ADB34B7EF4DF0E66EE66A9BEC6B
:109980005FF0006E060EE15C1200DECFE9FFDDCF76
:10999000EAFF12008DC2E9FF8EC2EAFF12003451C5
:1099A0000F0BE96EEA6AD890E936EA36120083C2F4
:1099B000E9FF84C2EAFF1200FCD8380EEE6E040EF6
:1099C000ED6E1200FD0EEA6ADB34BEEF4DF0FC0EC8
:1099D000DB50E824026EFD0EDB50040DF350022430
:1099E0001200DF50D7D8EA22EF6ADF50CED8EA2241
:1099F000EF6ADF2A1200E66EF4EC61F0006E050EED
:109A0000E15C1200EA22EE50EFCFEAFFE96E1200AD
:109A1000E66EA1C2E9FFA2C2EAFFA12B000EA223BB
:109A2000E552E750EF6EDF061200EA22EECFDEFFCE
:109A3000EDCFDDFF1200000EE66EE66AE66EE66A26
:109A4000120034510F0BC5EF4DF034510F0BCAEF1C
:109A50004DF0012200C0DEFF01C0DDFF1200FD0E4F
:109A6000DBCFE6FF1BEC49F0E552E5521200F7228E
:109A70000900F5CF95F20A00F5CF96F21200D95001
:109A8000020FE96E000EDA20EA6EEF501200160E99
:109A9000396F9F0E376F7B0E366F1200010EE66E28
:109AA000E66A000EE66EE66A1200F76A9525F66E23
:109AB0009651F722080012003251F66EF76AD890DC
:109AC000F636F736120085C2E9FF86C2EAFF1200B9
:109AD000040DF3CF00F0F4CF01F0000E0026040EC9
:109AE000B8DF840EDEEF4DF064D8300EEE6E040E5B
:109AF000ED6E1200020EE66EE66ADECFE6FFDDCF07
:109B0000E6FF050EBDEF4CF0E552E5CFDAFFE7CFFB
:109B1000D9FF1200020EE66EE66AE66A270EE66ECE
:109B20000F0EFBEF4CF01BDF8C0EEF6E33DF840E5D
:109B3000EF6E1200D9CFE6FFDACFE6FFE1CFD9FF13
:109B4000E2CFDAFF12002BDF870EE926020E1200A9
:109B500026DF8D0EE926020E12000ADF02EF4DF01D
:109B600014DFEF50800B1200FEDEE6521200FE0BF7
:109B7000EA36E96E8D0EE926020E1200FE0BEA3679
:109B8000E96E870EE926020E1200EA6AAB0FE96E53
:109B9000020E1200EA6AA80FE96E020E1200F5DE4C
:109BA000E850EF1612008FDFEE52400EEF6E63EFBB
:109BB0004DF0020EE926000EEA221200E6DEE85021
:049BC000EF1212008E
:0C9BC4001EEC53F0FB0EDBCFF3FFDB06C2
:109BD000F35000090AE06CEC53F0FA0ED7EC53F0A6
:109BE000F3E1011CF1E1010E01D0000E4DEF53F045
:109BF0001EEC53F03B0EE12402E3E168E652E16E15
:109C0000010EDB6A020EDB6AF90EDBCFF6FFFA0EFD
:109C1000DBCFF7FFFB0EDBCFF8FF0800F550DF6E60
:109C2000DF5002E171EF52F0250EDF5C02E064EFDD
:109C300052F0030EDB6A040EDB6A050EDB6A060EC9
:109C4000DB6A070EDB6A86EC52F02D0EDF5C0CE05F
:109C50002B0EDF5C09E0200EDF5C06E0230EDF5CEC
:109C600003E0300EDF5C1AE1DF50300A14E0130A23
:109C70000FE0030A0AE00B0A05E0060AE4E1030E1E
:109C8000DB80E1D7030EDB82DED7030EDB84DBD77C
:109C9000030EDB86D8D7030EDB88D5D72A0EDF5C10
:109CA0001BE182EC52F0D0EC52F010E0030EDB80AE
:109CB0003A683B68130EDBCF3FF0140EDBCF40F069
:109CC000BBEC56F0040E38C0DBFF03D0130EB9EC2A
:109CD00052F086EC52F00BD0090EDB6A27EC53F001
:109CE00003E09BEC53F0FAD7090EB9EC52F0030EE7
:109CF000DBB0DB982E0EDF5C1BE186EC52F02A0E07
:109D0000DF5C0BE182EC52F0D0EC52F003E1130E79
:109D10000BEC53F086EC52F00BD0090EDB6A27EC0B
:109D200053F003E09BEC53F0FAD7090E0BEC53F021
:109D3000680EDF5C07E186EC52F0680EDF5C1DE127
:109D4000030E18D0740EDF5C17E07A0EDF5C14E0AF
:109D5000480EDF5C06E0540EDF5C03E05A0EDF5C69
:109D600002E1020E07D06C0EDF5C03E06A0EDF5CDE
:109D700004E1010E5EEC53F0C9DBDF506E0A01E135
:109D80007FD31E0A01E192D1200A01E18FD13F0A5F
:109D900001E149D11A0A01E146D10D0A01E143D19D
:109DA000200A01E140D13A0A01E13DD1200A01E156
:109DB0003AD1260A01E135D10D0A01E132D11A0A60
:109DC00001E1D9D0200A4AE0300A1FE0460A0EE03D
:109DD000250A01E083D3D950F90FE96EFF0EDA208E
:109DE000EA6E010EEE5E000EEE5AEE5A6CEC53F087
:109DF000250EE66E95DB03E1011C01E169D368ECF9
:109E000053F001E26BD3DB2A69D3080EDB6A040E40
:109E1000DB50010806E2040EDB0430EC53F0DB50AB
:109E20008BDB080EDB5009E0030EDB50010B05E174
:109E300072DB01E04DD3080EDB6A64DBEFCFDFFF9E
:109E4000E0EC53F003E1011C01E142D368EC53F074
:109E500001E3DB2A60DB01E141D33AD3070EDB509B
:109E600002080FE1ACEC53F0030E73EC53F00E0E4E
:109E7000EECFDBFF0F0EEECFDBFF100EEECFDBFFE2
:109E800020D0F70EDBCF03F0F80EDBCF04F0020E8C
:109E9000035E000E045AF70E03C0DBFFF80E04C089
:109EA000DBFF03C0E9FF04C0EAFF63EC53F0026A82
:109EB0000E0E00C0DBFF0F0E01C0DBFF100E02C054
:109EC000DBFF0E0EDBCFE6FF0F0EDBCFE6FF100E43
:109ED000DBCFE6FF1CEC62F0E552E552E552130ED3
:109EE00039C0DBFF140E3AC0DBFF060EDB5005E085
:109EF000130EA7EC53F001E26ADBCBEC53F002E265
:109F0000130E37DB8EEC53F006E0040EA7EC53F093
:109F100002E2050E2EDB030EDBB005D0FCDA01E019
:109F2000D7D2080EDB6A090EDB6A0E0EDBCFF6FF16
:109F30000F0EDBCFF7FF100EDBCFF8FF0800F55058
:109F4000DF6EDF5014E0D1EC53F011E2E0EC53F09F
:109F500003E1011C01E1BCD2BBDB01E3DB2A090EFA
:109F6000DB2AD9500E0FE96E000ECBDBE7D7D3DA30
:109F700001E1B4D2ADD2C6DA110EEECFDBFF120E84
:109F8000EDCFDBFF110EDBCFE6FF120EDBCFE6FFDE
:109F90000EEC62F0E552E552130EF3CFDBFF140E28
:109FA000F4CFDBFF060EDB5004E0130ED0DB01E242
:109FB0000EDBCBEC53F002E2130EDBDAAFDB05E095
:109FC000040EC5DB02E2050ED4DA030EDBB005D0C9
:109FD000A2DA01E07DD2080EDB6A090EDB6A110EFF
:109FE000DBCFE9FF120EDBCFEAFFEFCFDFFFDF5061
:109FF00014E0D7DB12E2E4DB03E1011C01E168D2EB
:10A0000067DB01E3DB2A090EDB2A110EDB2ADBCF3B
:10A01000E9FF120EE8E3DB2AE6D77DDA01E15ED242
:10A0200057D2030EDB8E070EDB0410E195DB040E26
:10A030005ADB0A0EEECFDBFF0B0EEECFDBFF0C0E72
:10A04000EECFDBFF0D0EEECFDBFF6CD0070EDB504B
:10A0500003082CE1030EDBAE0DD0B2DA020E76DA85
:10A06000EFCF00F0016A026A036A00AE39D00168DE
:10A07000026835D0F70EDBCF01F0F80EDBCF02F02F
:10A08000020E015E000E025AF70E01C0DBFFF80E51
:10A0900002C0DBFF01C0E9FF02C0EAFFEFCF00F022
:10A0A0000A0E00C0DBFF0B0EDB6A38D0070EDB5058
:10A0B000020809E1030EDBAE04D059DB02AE10D07A
:10A0C0000ED055DB0DD0030EDBAE12D079DA020EC6
:10A0D0003DDAF9DA026A036A01AE02D00268036867
:10A0E000E2DA0C0E02C0DBFF0D0E03C0DBFF1AD05C
:10A0F000F70EDBCF02F0F80EDBCF03F0020E025EAC
:10A10000000E035AF70E02C0DBFFF80E03C0DBFFA0
:10A1100002C0E9FF03C0EAFFD6DAC5DA0C0EDB6A3B
:10A120000D0EDB6A060EDB5005E1010EF36E050E27
:10A13000F3CFDBFF150EDB6A160EDB6AD950370F43
:10A14000006E000EDA20016E390E00C0DBFF3A0E01
:10A1500001C0DBFF380EDB6A080EDB6A0A0EAEDADE
:10A16000DF50780A12E0200A10E0280A0CE0200AEA
:10A170000AE03F0A06E00D0A02E0200A08E1020EAA
:10A1800005D0080E03D0080EDF26100E97DA030E56
:10A19000DBBE02D0DB92DB94DB50800B24E08ADA5A
:10A1A000D890030EEB50000A08E6000EEE5C000E9D
:10A1B000EE58000EEE58000EEE5815E213DA3D6828
:10A1C0003E683F68406817EC63F00A0E34C0DBFF5E
:10A1D0000B0E35C0DBFF0C0E36C0DBFF0D0E37C09B
:10A1E000DBFF2D0E08D0030EDBA202D02B0E03D016
:10A1F000DBA408D0200EF36E170EF3CFDBFF150E95
:10A20000DB2A02D0170EDB6A050EDB5003E1B7D95B
:10A2100001E189D0020E006EC80E016E000E026EC2
:10A22000070EDBCF03F0046A056A066A03C03DF03F
:10A2300004C03EF005C03FF006C040F0D3D975EC35
:10A2400063F000503424F36E01503520F46E025058
:10A250003620F86EF4CFF7FFF3CFF6FF0800090EB3
:10A26000F5CFDBFF580EDF5C0FE1610EF36E090ED8
:10A270007BD90AE3200E006E090EDBCFE7FF00500A
:10A28000E75E090EE7CFDBFF070EDBCF00F0016AC8
:10A29000026A036A0FDA00C03DF001C03EF002C05E
:10A2A0003FF003C040F0EECF38F0EECF39F0EECF04
:10A2B0003AF0EFCF3BF075EC63F03BC0EDFF3AC0F6
:10A2C000EDFF39C0EDFF38C0EFFF390EDBCFE9FFFE
:10A2D000DB063A0EDBCFEAFF01E2DB06090EDBCF3D
:10A2E000EFFF150EDB2A4BD995E1030EDBA61DD03F
:10A2F0006F0EDF5C06E1C1D918E3150EDB285BDACF
:10A3000014D0780EDF5C09E0580EDF5C06E0620EC8
:10A31000DF5C03E0420EDF5C08E1020EF36E160E16
:10A32000F3CFDBFF02D0150EDB6A030EDB50100B00
:10A330000EE0040EDBCF00F0050EDB50D880005499
:10A3400006E2060EDB5003E1040EDB5034DA95D949
:10A350000AE2050EDBCFE7FF150EDB50E75E050EC8
:10A36000E7CFDBFF02D0050EDB6A040EDBCF00F087
:10A37000160E45D9D880005414E2160EDBCFE6FF46
:10A38000150EDBCFE6FF040EDBCFE6FF050EDB503C
:10A39000E552E75CE552D880E754E552D880E754AF
:10A3A0005FD9030EDB50010B0BE1080EDB5008E018
:10A3B000B2D801E08DD0080EDB50BED8080EDB6AA3
:10A3C000170EDB5007E088D9170EF1D903E1011C05
:10A3D00001E17ED0160EDB5016E07ED9300EE66E1F
:10A3E0009FD802E1011C74E077D9DFCFE6FFD5ECFE
:10A3F00062F0E552E552E552F4CF01F00001F31CA2
:10A4000002E1011C65E0050EDBCF00F0160EDB500B
:10A41000D880005409E2050EDBCFE7FF160EDB50B3
:10A42000E75E050EE7CFDBFF300EE66E050ECBD9FB
:10A430004FE1390EDB2ADBCFE9FF3A0E01E3DB2ADD
:10A44000DBCFEAFF090EEFCFDBFFDB500EE044D994
:10A45000090EADD902E1011C3BE0390EDB2ADBCF4E
:10A46000E9FF3A0EEDE3DB2AEBD755D831E1160EC2
:10A47000DBCFE6FF080EC3D8E552E7245DD82ED027
:10A48000070EDB50030A1CE0010A14E0030A07E090
:10A490007BD9DBCFEEFF020EDBCFEDFF1FD0F5D86F
:10A4A000056A03AE02D0046805682CD8BCD805C084
:10A4B000EEFF14D0EAD803BE046824D8B4D80ED076
:10A4C00063D9DBCFEFFF0AD07BD905E1011C03E1A3
:10A4D000F368F46810D0FCD801E3DB2A79D90DEFDA
:10A4E0004EF0010EDBCF00F0020EDBCF01F000C01A
:10A4F000F3FF01C0F4FF3B0EE15C02E2E16AE552CA
:10A50000E16ECBD029D9020E73EF53F061D9080068
:10A51000F550DF6E1200200EE66E080EE3EF53F0EA
:10A52000D5EC62F0E552E552E552F3CF00F0F4CFFE
:10A5300001F00001F31C1200006E016AD950010FF6
:10A540004DD90050EE260150ED221200045E000E9F
:10A55000055AF70E04C0DBFFF80E05C0DBFF04C090
:10A56000E9FF05C0EAFF1200DBCFF4FFF350F45C13
:10A570001200DB50E76E040EE7CFDBFF12000A0E7D
:10A58000DBCF00F00B0EDBCF01F00C0EDBCF02F0C7
:10A590000D0EDBCF03F0005001100210031012006B
:10A5A000130EEECFDBFF140EEDCFDBFF130EDBCF70
:10A5B00000F0140EDBCF01F00001800E0114120038
:10A5C000F70EDBCF04F0F80EDBCF05F01200050E1E
:10A5D000DB50E66ED950130F01D9E552E750EE6E0D
:10A5E000ED6A12000A0EDBCF38F00B0EDBCF39F02C
:10A5F0000C0EDBCF3AF00D0EDBCF3BF01200DBCFC1
:10A60000E6FF150EDBCFE6FF050EDB50E552E72433
:10A61000E552E7241200DB50CED8010EF36E060E91
:10A62000F3CFDBFF1200EE50EFCFEAFFE96E02C07E
:10A63000EEFF03C0EEFF04C0EEFF1200D9CFE6FF2D
:10A64000DACFE6FFE1CFD9FFE2CFDAFF1200DFCFAA
:10A65000E6FFE66A63EC63F0E552E552F350120060
:10A66000E76E080EE7CFDBFF1200EECF00F0EECF73
:10A6700001F0EFCF02F0036A1200050EDBCF00F00D
:10A68000150EDB50D88000541200010EDBCF02F013
:10A69000020EDBCF03F0046A1200E552E5CFDAFFC9
:10A6A000E7CFD9FF12000A0E00C0DBFF0B0E01C07E
:10A6B000DBFF1200D9500A0FEEEF53F0F36E070ED6
:10A6C000F3CFDBFF1200EECF00F0EFCF01F012006E
:10A6D000010EDB2A020E1200FC0EDBCFE6FFFD0EA0
:10A6E000DBCFE6FF1200005E000E015AF70E00C03D
:10A6F000DBFFF80E01C0DBFF00C0E9FF01C0EAFF8D
:10A700001200DA20EA6EEF2AEECFF6FF000EEF22FB
:10A71000EECFF7FFEF22EECFF8FF1200040EDBCFF3
:10A72000E6FF130EDB50E552E75C9ADFDB5004DFF7
:10A73000060EDB501200090EDB500A0DF350DF2429
:10A74000D00FE76E090EE7CFDBFF86EF52F0DB504C
:10A75000F36E050EB4EF52F0F70EDBCF00F0F80EFB
:10A76000DBCF01F01200DFCFE6FF90EF52F028DFE1
:10A77000030EECDE35EF53F0E2EC4DF0E552E5521E
:10A78000E552E55200091200BDDEEE50EFCFEAFFC0
:10A79000E96E010E1200130EDB50F36E040EB4EFDF
:10A7A00052F0040EDB50F36E090EB4EF52F0DBCF23
:10A7B000E6FF90EF52F0E76E050EE7CFDBFF1200E9
:10A7C0008BDFB3EF53F0DBCFE6FF86DFBCEF53F058
:10A7D000D950F90FE96EFF0E81EF53F0E96E000ECC
:06A7E000DA20EA6E12000F
:0AA7E600439E08D0439E3BAE05D011
:10A7F0003A6C3B1EE86A3B22438E3BC035F03AC0C0
:10A8000034F0476A466A8E0E366E376ACDEF55F0E1
:10A81000439E0CD0439E3BAE09D0386C391E3A1E85
:10A820003B1EE86A39223A223B22438E3BC035F078
:10A830003AC034F039C047F038C046F09E0E366E4C
:10A84000376ACDEF55F0436A09EC56F021EC56F02B
:10A8500043B6B1EF55F043A205D043BAB1EF55F07E
:10A86000B8EF55F043BAC4EF55F043A005D043B854
:10A87000B1EF55F0C4EF55F043B8B8EF55F0376A73
:10A880007F0E3C24366EE86A37224150365EE86A15
:10A89000375A1A0E446E3C6A466A476A346A356A09
:10A8A0003E50395E3F503A5A40503B5A000E3C5A97
:10A8B00009E73E5039263F503A2240503B22000ED5
:10A8C0003C2201D0468AD89039363A363B363C365F
:10A8D000D8904636473634363536442EE1D73B508D
:10A8E0003A103910D8A4468ACDEF55F0436A09ECE6
:10A8F00056F021EC56F043B6B1EF55F043A205D027
:10A9000043B8B1EF55F0B8EF55F043AA05D043B0C6
:10A91000B1EF55F0B8EF55F043B002D043A802D0E4
:10A92000C4EF55F0376A41503C24366EE86A37224E
:10A930007E0E365EE86A375A466A476A346A356A76
:10A9400040503B02F4CF35F0F3CF34F03F503B02A0
:10A95000F3504726F4503422000E352240503A027C
:10A96000F3504726F4503422000E35223E503B026D
:10A97000F3504626F4504722000E342235223F5031
:10A980003A02F3504626F4504722000E3422352274
:10A9900040503902F3504626F4504722000E34222C
:10A9A00035223E503A02F4504626000E4722342209
:10A9B00035223F503902F4504626000E47223422F9
:10A9C0003522CDEF55F0417E436A09EC56F021EC7B
:10A9D00056F043B6B1EF55F043A20AD043AA03D0D4
:10A9E00043BEB1EF55F043A4BDEF55F0BAEF55F0BB
:10A9F00043AA05D043ACBDEF55F0BAEF55F043A0E4
:10AA00000AD043A808D043BE04D043A402D0C6EF66
:10AA100055F0CAEF55F0466A376A41503C5C456EC6
:10AA200010E339C047F03AC034F03BC035F03CC0C9
:10AA300044F03EC039F03FC03AF040C03BF0433AEA
:10AA400009D03EC047F03FC034F040C035F041C0AF
:10AA500044F0456C439E43BC438E44C036F043B043
:10AA6000F9EF55F01A0E4560F9EF55F0366A3C6A79
:10AA700043A408D0396C3A1E3B1E3C1EE86A3A22B9
:10AA80003B223C2243AC08D0476C341E351E361E98
:10AA9000E86A342235223622386A455207E03C34CF
:10AAA0003B323A3239323832452EF9D739504726BF
:10AAB0003A5034223B5035223C50362238C046F0C2
:10AAC000439E36AE0BD0466C471E341E351E361ED6
:10AAD000E86A4722342235223622438E36A006D039
:10AAE000D8803532343247324632442A44C036F0B8
:10AAF000CDEF55F0436A09EC56F043B684EF55F0BC
:10AB000043A20FD043B407D07F0E3B6EFF0E3A6EC8
:10AB1000396E386E25D0800E3B6E01D03B6A000E38
:10AB2000F6D743B0FBD7386A9F0E3C60EBD77E0E5A
:10AB30003C64F4D79E0E3C5C07E0D8903B323A323E
:10AB4000393238323C2AF6D743A40AD0386C391E41
:10AB50003A1E3B1EE86A39223A223B223BAEDED740
:10AB600012007F0E3C6EFF0E3B6E3A6E396E120085
:10AB70007F0E43BEFF0E3C6E02D07F0E3C6E800EF9
:10AB80003B6E3A6A396AF3D743AE04D0800E3C6E0E
:10AB90003B6AF7D73C6A3B6AF4D73550341047100C
:10ABA0004610F8E037BEF0D735BE0CD0365037101F
:10ABB000EBE0D89046364736343635363606D8A0E0
:10ABC0003706F2D73750D4E13628D2E046AE11D05E
:10ABD0007F0E461402E147A00CD0472AE86A3422CF
:10ABE000352207E3D880353234324732362A3628C8
:10ABF000BFE03650C9E047C039F034C03AF03534D0
:10AC00003B6E36303C6E3B323C9E43BE3C8EB7EFD3
:10AC100055F03B363C3602E34384437E06E14380F5
:10AC20003C6A3B6A3A6A396A12003C2803E0D880E1
:10AC30003B321200D8903B3202E14382120043863D
:10AC400012004036413602E3438C437E06E14388DE
:10AC5000416A406A3F6A3E6A1200412803E0D88098
:10AC600040321200D8904032EAE1438A1200426A30
:10AC700040AE40EF56F03F6C401EE86A4022421E54
:10AC80003BAE48EF56F03A6C3B1EE86A3B22421E50
:10AC9000B4EC63F03BBE58EF56F042AE000C3A6C99
:10ACA0003B1EE86A3B22366C371EE86A3722000CEE
:10ACB00042BE4FEF56F04388FF0C66EC56F043B6A9
:10ACC000000C43B0000C43A4000C010C436A09ECD7
:10ACD00056F021EC56F043B6120043AE08D043A024
:10ACE00004D043A802D04380120043901200415088
:10ACF0003C5C0BE140503B5C08E13F503A5C05E1B5
:10AD00003E50395C02E143801200D8A002D0438E4D
:10AD100010D03C5041C03CF0416E3B5040C03BF035
:10AD2000406E3A503FC03AF03F6E39503EC039F065
:10AD30003E6E41503C5C10E0FF0F09E0439043B48D
:10AD400003D043AE4384120043AE43941200412A21
:10AD5000D89040323F323E323E50395E3F503A5AF0
:10AD600040503B5A3BBEEAD7D89039363A363B364C
:10AD70003C2EF8D7C8D73BC047F03AC046F03A500F
:10AD80003F02F4CF39F0F3CF38F03B504002F4CF1C
:10AD90003BF0F3CF3AF03F02F3503926F4503A2219
:10ADA000E86A3B2246504002F3503926F4503A22DA
:10ADB000E86A3B2240AEE1EF56F046503A5E47501B
:10ADC0003B5A47AE000C3F503A5E40503B5A000C95
:10ADD000256C692C256C690A0D00514D2C25692CB8
:10ADE00025692C25692C25690A0D00253034692C2C
:10ADF000253034690D0A002531690D0A00253033EC
:10AE0000690D0A00253031306C750D0A0025640A81
:10AE10000D0025642C256C752C256C752C256C7506
:10AE20002C256C750A0D004D616A6F72206D616C86
:10AE300066756E6374696F6E204178697332205352
:10AE4000746570436F756E746572207A65726F0AEF
:10AE50000D004D616A6F72206D616C66756E637472
:10AE6000696F6E2041786973322053746570436F47
:10AE7000756E74657220746F6F2068696768203A18
:10AE800020256C750A0D004D616A6F72206D616C32
:10AE900066756E6374696F6E2041786973312053F3
:10AEA000746570436F756E746572207A65726F0A8F
:10AEB0000D004D616A6F72206D616C66756E637412
:10AEC000696F6E2041786973312053746570436FE8
:10AED000756E74657220746F6F2068696768203AB8
:10AEE00020256C750A0D002130204572723A203CF5
:10AEF00061786973323E2073746570207261746585
:10AF0000203C20312E3331487A2E0A0D002130208A
:10AF10004572723A203C61786973323E20737465E1
:10AF2000702072617465203E2032354B2073746549
:10AF300070732F7365636F6E642E0A0D00213020CD
:10AF40004572723A203C61786973313E20737465B2
:10AF5000702072617465203C20312E3331487A2E86
:10AF60000A0D002130204572723A203C61786973E5
:10AF7000313E20737465702072617465203E20320A
:10AF8000354B2073746570732F7365636F6E642E19
:10AF90000A0D002130204572723A203C6D6F7665B3
:10AFA0005F6475726174696F6E3E206C6172676573
:10AFB00072207468616E2031363737373231352070
:10AFC0006D732E0A0D002130204572723A203C61CB
:10AFD000786973323E20616363656C657261746980
:10AFE0006F6E2076616C756520697320302E0A0DB6
:10AFF000002130204572723A203C61786973313EFD
:10B0000020616363656C65726174696F6E2076613F
:10B010006C756520697320302E0A0D0021302045A3
:10B0200072723A203C61786973323E206C617267BB
:10B030006572207468616E203136373737323135AA
:10B040002073746570732E0A0D00213020457272D2
:10B050003A203C61786973313E206C617267657299
:10B06000207468616E2031363737373231352073BE
:10B07000746570732E0A0D002130204572723A20DB
:10B080003C76656C6F636974795F66696E616C3E6E
:10B09000206C657373207468616E20342E0A0D0075
:10B0A0002130204572723A203C76656C6F6369747A
:10B0B000795F696E697469616C3E206C6573732099
:10B0C0007468616E20342E0A0D00213020457272A2
:10B0D0003A203C76656C6F636974795F66696E616E
:10B0E0006C3E206C6172676572207468616E2032FC
:10B0F000353030302E0A0D002130204572723A2052
:10B100003C76656C6F636974795F696E69746961B7
:10B110006C3E206C6172676572207468616E2032CB
:10B12000353030302E0A0D005374617475733D252F
:10B13000690D0A002135204572723A204E6565641A
:10B1400020636F6D6D61206E6578742C20666F755D
:10B150006E643A20272563270D0A00506172616DE5
:10B16000383D25630D0A00506172616D373D2563DE
:10B170000D0A00506172616D363D256C750D0A0037
:10B18000506172616D353D256C640D0A005061722D
:10B19000616D343D25750D0A00506172616D333D5E
:10B1A00025640D0A00506172616D323D25640D0AFF
:10B1B00000506172616D313D25640D0A0050492CCB
:10B1C0002531750D0A004D522C253033750D0A00BE
:10B1D0002C253032753A25303475004100492C2534
:10B1E0003033692C253033692C253033692C2530D8
:10B1F00033692C253033690D0A00213820457272DD
:10B200003A20556E6B6E6F776E20636F6D6D616E59
:10B21000642027256325633A253258253258270DA7
:10B220000A002138204572723A20556E6B6E6F7796
:10B230006E20636F6D6D616E64202725633A253241
:10B2400058270D0A002137204572723A204578743C
:10B250007261207061726D617465720D0A00213631
:10B26000204572723A20496E76616C696420706183
:10B2700072616D7465722076616C75650D0A0021CE
:10B2800034204572723A204D697373696E6720707D
:10B290006172616D657465722873290D0A0021332E
:10B2A000204572723A2052582042756666657220B7
:10B2B0006F76657272756E0D0A00213220457272CA
:10B2C0003A20545820427566666572206F76657222
:10B2D00072756E0D0A002131204572723A20436169
:10B2E0006E277420737465702074686174206661C1
:10B2F00073740D0A002130200D0A00200800257308
:0DB30000001B5B421B5B314B1B5B304700A9
:02B30E00D9CF95
:10B31000E6FFDACFE6FFE1CFD9FFE2CFDAFF240E76
:10B32000E12402E3E168E652E16ED950FA0FE96EDA
:10B33000FF0EDA20EA6E020EEECFDBFF030EEECF39
:10B34000DBFF040EEECFDBFF050EEECFDBFFE8D90F
:10B35000F2D98AEC60F0006E060EE15C02E2E16A6E
:10B36000E552E16E0050E76E0D0EE7CFDBFFDB50DC
:10B37000800815E0A0D93E6A3F6A406A416A00C071
:10B3800039F001C03AF002C03BF003C03CF05DEC84
:10B3900056F0010A10E1210E0701F16FF26B020E67
:10B3A000DB68030EDB68040EDB687F0EF36E050EB0
:10B3B000F3CFDBFF66D10D0EDB50050B01E061D151
:10B3C0000A0EDBCF00F00B0EDBCF01F0830E002660
:10B3D000FF0E012200C0DEFF01C0DDFFD950060FC5
:10B3E00065D976D9DF50010B0FE0DF06010E01E2CF
:10B3F000DB06D950180F5AD9D890EF36010EEB362C
:10B40000020EEB36030EEB36D9CFE9FFDACFEAFFB7
:10B41000020E3F6E406AEECF3AF0EDCF3BF037ECD4
:10B4200056F03AC0EEFF3BC0EDFF140EDB6A150E7E
:10B43000DB6A160EDB6A170EDB6A1C0EDB6A1D0E5A
:10B44000DB6A1E0EDB6A010EF36E1F0EF3CFDBFF0D
:10B45000010EF36E0E0EF3CFDBFF0F0EDB6A0E0E46
:10B46000DBCF00F00F0EDBCF01F0D890015004E6E7
:10B470001A0E005C000E015801E398D0180EDBCFC5
:10B4800000F0190EDBCF01F01A0EDBCF02F01B0E1D
:10B49000DBCF03F0010E1F0B07E0D890003601361A
:10B4A00002360336E806F9E1180E00C0DBFF190E7C
:10B4B00001C0DBFF1A0E02C0DBFF1B0E03C0DBFF67
:10B4C000140EDBCF08F0150EDBCF09F0160EDBCF24
:10B4D0000AF0170EDBCF0BF0010E1F0B07E0D89020
:10B4E000083609360A360B36E806F9E1D9501C0F42
:10B4F000DDD80850EE24046E0950EE20056E0A5087
:10B50000EE20066E0B50EE20076ED950180FCED8E5
:10B510000450EE5C006E0550EE58016E0650EE5879
:10B52000026E0750EE58036E200E00C0DBFF210EA6
:10B5300001C0DBFF220E02C0DBFF230E03C0DBFFD6
:10B54000200EDBCF39F0210EDBCF3AF0220EDBCF1D
:10B550003BF0230EDBCF3CF03C34000E3C1809E6F8
:10B56000D880000E3954000E3A54000E3B54000EA1
:10B570003C5411E2D950200F99D8AAD8D8D81C0E23
:10B58000DB50EE121D0EDB50EE121E0EDB50EE12E3
:10B590001F0EDB50EE12D9501C0F88D8AFD80E0EFC
:10B5A000DB2A0F0E01E25BD7DB2A59D7C9D8100E70
:10B5B00000C0DBFF110E01C0DBFF180EDBCF3AF03D
:10B5C000190EDBCF3BF0120E3AC0DBFF130E3BC06F
:10B5D000DBFFADD893D8D950100F68D8EE50ED10DE
:10B5E00012E0D950120F62D8EE50ED1006E1A8D843
:10B5F000005001100210031006E099D8EE2A000E48
:10B60000EE22EE22EE220C0EDB6A91D8060EEECF71
:10B61000DBFF070EEECFDBFF080EEECFDBFF090EE0
:10B62000EECFDBFF7E0EF36E0A0EF3CFDBFF0B0EC9
:10B63000DB6AD950020FE66E000EDA20E66E70D893
:10B6400018EC61F0E552E552E552E552DECFE6FF37
:10B65000DDCFE6FF70D8EEEC5FF0006E060EE15C29
:10B6600002E2E16AE552E16E0050020E38C0DBFFF3
:10B67000030E39C0DBFF040E3AC0DBFF050E3BC0F2
:10B68000DBFF19D800C038F001C039F002C03AF031
:10B6900003C03BF0240EE15C02E2E16AE552E16E98
:10B6A000E552E5CFDAFFE7CFD9FF1200E96E000ED1
:10B6B000DA20EA6E1200020EDBCF00F0030EDBCFC1
:10B6C00001F0040EDBCF02F0050EDBCF03F0120019
:10B6D000180EEECFDBFF190EEECFDBFF1A0EEECF0A
:10B6E000DBFF1B0EEECFDBFF1200EECFE6FFEECF4F
:10B6F000E6FFEECFE6FFEFCFE6FF1200D890030E95
:10B70000EB32020EEB32010EEB32EF321200EE5052
:10B710000016EE500116EE500216EE5003161200FF
:10B72000D950060FE66E000EDA20E66E1200D950F0
:10B73000140F56EF5BF0D950020FB8DF75EF5BF0D6
:10B74000010E006E016A026A036AF1DF87EF5BF0A7
:10B75000040130511F0B010801E012003051600B51
:10B76000E842E842E842E842E842010801E012000B
:10B77000345103E0340501E012003151220A31E076
:10B78000030A24E0010A15E0210A0DE0010A01E0A4
:10B7900012000201A00E956F070E966F080E986FAB
:10B7A000996B978121D00201A00E956F070E966FBD
:10B7B0001BD036C49DF237C49EF20201800E9A6FF0
:10B7C000070E9B6F9F6BA06B9C8F12000201800E77
:10B7D000956F070E966F070E986F996BC10E976F56
:10B7E000120032C49BF70201978F12000701806B91
:10B7F0004B0E816F826B836B846B856B080E866F3B
:10B800008F6B1A0EE66E010EE66E44EC48F0E552C0
:10B81000E5521E0EE66E020EE66E44EC48F0E5526E
:10B82000E5522FD902E2E16AE5524FD90701996B3F
:10B830009A6B906B12001CD982D9050E3A1801E15F
:10B840003B5002E0000E18D051D907019751001863
:10B8500008E19851011805E114D902E2E16AE552C4
:10B8600034D944D907019951001805E19A510118BA
:10B8700002E1906B956B010E0CD1FAD807018F6B2A
:10B880009751981102E1000E05D045D9EF50800B79
:10B8900001E0010E000931E1FB0EDBCF00F03BD9E6
:10B8A000EE52EF50D880005405E235D9EE52FB0E2F
:10B8B000EFCFDBFF8F6BFB0EDB508F5D19E28F51FB
:10B8C000EA6A400FE96E070EEA22EF50E66E8F51EA
:10B8D000E76EFC0EDBCFE9FFFD0EDBCFEAFFE750A2
:10B8E000E926000EEA22E552E750EF6E8F2BE3D7F0
:10B8F000C8D802E2E16AE552E8D807018F51C9D001
:10B90000B7D80701905107E1E7D8FB0EDBCF95F7D9
:10B91000010E966F906FBDD00BD917E1C0D8EDD84E
:10B9200002E101500BE0010EDBCFE9FFDB2A020E42
:10B93000DBCFEAFF01E3DB2AEF50F1E1CDD8DFCF27
:10B9400095F70701010E966F906FE552E552E552AB
:10B95000A0D0EED818E1A3D8D0D802E101500CE075
:10B96000010EDBCFF6FFDB2A020EDBCFF7FF01E390
:10B97000DB2A0800F550F0E1AFD8DFCF95F70701DB
:10B98000966B010E906FE552E552E55282D070D869
:10B99000E652E652070199519A1102E1000E08D0D1
:10B9A00099C7E9FF9AC7EAFFEF50800B01E0010E4B
:10B9B00000095BE1030E905D01E1906B905155E051
:10B9C000020E905D0DE1E66A000EE66EE66A8BD827
:10B9D00002E2E16AE55298D80701030E906F45D064
:10B9E000900543E1400E006E016A9551005C000E27
:10B9F000015803E2400EDF6E02D095C7DFFFDF5033
:10BA0000955D956F000E936F070E946F010EDFCF5B
:10BA1000DBFF96510BE1010EDB5012E091C7F6FF00
:10BA200092C7F7FF0800F55043D8F5D7010EDB5059
:10BA300007E091C7E9FF92C7EAFFEF5039D8F6D780
:10BA40000701955107E1400EDF5C02E1020E01D0D3
:10BA5000030E906FDFCFE6FF000EE66E070EE66E78
:10BA600042D802E2E16AE5524FD8E552E55211D0E0
:10BA7000D9CFE6FFDACFE6FFE1CFD9FFE2CFDAFF99
:10BA80001200400EE66E400EE66E070EE66EE66AA7
:10BA900047D0E552E5CFDAFFE7CFD9FF1200DF6AE2
:10BAA0004ED8DE523AC0DEFF3BC0DDFFDD52120051
:10BAB00093C7E9FF94C7EAFFEF6E932B000E942320
:10BAC000912B9223010EDB061200E16E0050F3CFA2
:10BAD00097F7F4CF98F71200FC0EDBCF91F7FD0E2D
:10BAE000DBCF92F71200010EE66E1AD0FA0EDBCF12
:10BAF00000F0FB0EDBCF01F01200DF2ADF50006EFA
:10BB0000016AFF0E00181200E16E0050F3CF99F7A2
:10BB1000F4CF9AF7120097C7E9FF98C7EAFF12001F
:10BB2000020EE66E63EC48F0006E050EE15C12005A
:10BB30009FDFE652E652E652070190511200FC0EDA
:0CBB4000DBCF3AF0FD0EDBCF3BF0120033
:04BB4C006AD9E6527A
:10BB50000E01006BA96BDF6A180EDF5C14E283D95B
:10BB6000010EE9260E0E85D9DF5077D9EF6A7BD911
:10BB7000490EE9260E0E7DD976D9790EE9260E0EEC
:10BB800078D9DF2AE9D70E01C60EAC6F0E0EAD6F65
:10BB90003F0E79140009796ECF0E79140009796E81
:10BBA00079827B6A7A6A79900F0152815293F00E02
:10BBB000B4140909B46E0E01080EAA6F030EAB6F20
:10BBC000800EAE6F3E0EAF6FE00EB06F2E0EB16FF7
:10BBD000040EB66F900EB26F010EB36F900EB46F7D
:10BBE000010EB56F000EE66EE66A010EE66E7CECA5
:10BBF0002FF0E552E552E552E55229D112D9E6522D
:10BC0000DF6A180EDF5C0AE2DF5027D9EFCF00F0C1
:10BC1000FD0EDB50005C0AE0DF2AF3D7DF6A180E66
:10BC2000DF5C08E2DF5019D9EF5002E1DF2803D0D2
:10BC3000DF2AF5D7000EE5520AD1F3D8070EE1242A
:10BC400002E3E168E652E16EDE6ADD6A020EDB6A5B
:10BC5000030EDB6A040EDB6A050EDB6A060EDB6A86
:10BC6000010EE66ED9CFE6FFDACFE6FF030EE2D88B
:10BC7000020F03D9010EDED8030FFFD8030EDAD866
:10BC8000050FFBD8030EFED80701B45124E1020EC4
:10BC9000DB50180802E2B48D1ED0050EDBCFE6FFA4
:10BCA000060EDBCFE6FF030EDBCFE6FF040EDBCF95
:10BCB000E6FF020EDBCFE6FFDECFE6FFDDCFE6FFDD
:10BCC00011D8006E070EE15C02E2E16AE552E16E16
:10BCD00000500EEC3DF0070EE15C02E2E16AE55235
:10BCE000E16EB5D09ED8E652E652FB0EDBCFE6FF02
:10BCF00085DFE552E76E010EE7CFDBFFDB5002E1A7
:10BD0000000E8CD0D950FC0FE96EFF0EDA20EA6EDF
:10BD1000EE50ED101FE1010EDB049FD8EF500E0135
:10BD2000EA6AAC25E96EAD51EA22EF6A88D8790E4D
:10BD3000E9260E0E9ED883D8490EE9260E0E99D814
:10BD4000010EDB048AD8EF6A7AD8010EE9260E0EBE
:10BD500090D862D0010EDB04006E0E01AA51005C87
:10BD60005BE2FB0EDB50180857E3FB0EDB500708C5
:10BD700002E10601CF6B63D8010EE9260E0EEA221E
:10BD8000EE50ED1010E1E66AFB0EDBCFE6FFD0ECE3
:10BD900044F0E552E552E66AFB0EDBCFE6FFA2EC8B
:10BDA00044F0E552E55206012351FDE00601030E81
:10BDB000306FF70EDBCF46F6F80EDBCF47F6486B59
:10BDC000496B190E3D6E3E6A3F6A406A46C638F0BE
:10BDD00047C639F048C63AF049C63BF017EC63F065
:10BDE00034C046F635C047F636C048F637C049F687
:10BDF000010EDBCF4DF6FB0EDBCF4CF6FC0EDBCF9E
:10BE00004AF6FD0EDBCF4BF6F90EDBCF4EF6FA0EFF
:10BE1000DBCF4FF60601236B010EDB50E552E552F6
:10BE200016D0D9CFE6FFDACFE6FFE1CFD9FFE2CFD8
:10BE3000DAFF120027D8010EE66ED9501200010E6B
:10BE4000DB04E96EEA6AD890E936EA361200E55278
:10BE5000E5CFDAFFE7CFD9FF1200EA6A310FE96ECA
:10BE60000E0EEA221200EA6ADF34FE0BEA36E96EB1
:10BE70001200EA22EE6AED6A1200E66E000EDA2087
:10BE8000E66E1200E66E6DEC42F0E552E552E552C8
:04BE9000E552120065
:0CBE940005D886EC47F0CDEC38F0FBD769
:10BEA0008ED8E652E6520F0148694969600ED36E9A
:10BEB0009B8C580EDE6E020EDD6EDFCF00F0DF06CB
:10BEC000010EDBCF01F001E2DB0600500110F5E1CD
:10BED000948E40EC38F01CEC47F0E552E55278D0F7
:10BEE0001200120012001200A8EF5BF01200F6EF31
:10BEF0005BF00201A3051EE10201A4051BE1F1DFD5
:10BF000065920201A46B0701100EEF6F0E0EF06F29
:10BF1000EF07000EF05BEF51F011FAE16584080EB7
:10BF2000EF6F070EF06FEF07000EF05BEF51F011AF
:10BF3000FAE16594120043D8FC0EDBCF3AF0FD0E17
:10BF4000DBCF3BF0050E3A1801E13B5036E0E868E4
:10BF50003A1802E17F0E3B182FE0030E3A1801E178
:10BF60003B5028E0020E3A1801E13B5021E0010E5F
:10BF70003A1801E13B501AE0740E3A1801E13B50C7
:10BF800013E0750E3A1801E13B500CE0730E3A18BD
:10BF900001E13B5005E0720E3A180FE13B500DD025
:10BFA000A1DF0BD09DDF09D09CDF07D0A0DF05D03B
:10BFB0009DDF03D099DF01D096DF010E09D0D9CFE4
:10BFC000E6FFDACFE6FFE1CFD9FFE2CFDAFF1200DA
:0CBFD000E552E5CFDAFFE7CFD9FF120001
:04BFDC0096D8E1CF43
:10BFE000D9FFE2CFDAFF0C0EE12402E3E168E6526A
:10BFF000E16ED950FA0FE96EFF0EDA20EA6E080EF4
:10C00000EECFDBFF090EEECFDBFF0A0EEECFDBFF3C
:10C010000B0EEECFDBFF79D8D950080FE96E000E7A
:10C02000DA20EA6EEECFE6FFEECFE6FFEECFE6FFD8
:10C03000EFCFE6FF8AEC60F0006E060EE15C02E2F4
:10C04000E16AE552E16E0050E76E070EE7CFDBFFD5
:10C05000DB50840B3AE1070EDB041AE1060EDB50DD
:10C0600006E0006A016A026A800E036E04D0006A6C
:10C07000016A026A036A080E00C0DBFF090E01C0F4
:10C08000DBFF0A0E02C0DBFF0B0E03C0DBFF1DD07F
:10C09000F80EDBCF00F0F90EDBCF01F0D950040F22
:10C0A000E96E000EDA20EA6E0050EE260150ED2215
:10C0B000D950080FE66E000EDA20E66E26D818EC8E
:10C0C00061F0E552E552E552E552080EDBCF00F093
:10C0D000090EDBCF01F00A0EDBCF02F00B0EDBCF37
:10C0E00003F000C038F001C039F002C03AF003C0DC
:10C0F0003BF00C0EE15C02E2E16AE552E16EE552D2
:10C10000E5CFDAFFE7CFD9FF1200D9CFE6FFDACFCC
:04C11000E6FF120034
:0CC11400D9CFE6FFDACFE6FFE1CFD9FF7C
:10C12000E2CFDAFFE652006801687F0E026E036A12
:10C13000D950FA0FE96EFF0EDA20EA6EEE500016C3
:10C14000EE500116EE500216EE5003166AD800C0EB
:10C15000EEFF01C0EEFF02C0EEFF03C0EEFFFD0EDA
:10C16000DB50800B02E0010E01D0000EE66E59D8C4
:10C17000060EE926000EEA22E552E750EF6EFC0EAD
:10C18000DBCF00F0FD0EDBCF01F0D890003601369A
:10C19000FC0E00C0DBFFFD0E01C0DBFFDB50E66ED6
:10C1A00040D8040EE926000EEA22E552E750EE6E72
:10C1B000ED6AFD0EDB50006E016AFF0E001818E1FB
:10C1C000015016E12ED8EECF00F0EECF01F0EECF09
:10C1D00002F0EFCF03F0005001100210031006E050
:10C1E000210E0701F16FF26B800E0BD0040E09D007
:10C1F000FD0EDB5008E115D8EE6AEE6AEE6AEE6AD3
:10C20000010EDF6E06D0020EDF6E0BD8EE52EE523C
:10C21000EE8EDF50E552E552E5CFDAFFE7CFD9FFEA
:10C220001200F80EDBCFE9FFF90EDBCFEAFF1200B8
:10C23000D9CFE6FFDACFE6FFE1CFD9FFE2CFDAFFD1
:10C240005BD8013411E20050FE08000E01540CE2EC
:10C2500076D805E06CD8800EEE6EEE6847D067D8D1
:10C26000800EEE6E7F0E0ED047D8D890015004E6B7
:10C27000010E005C000E01580BE261D805E057D8B2
:10C28000EE6A800EEE6E32D052D8EE6AEE6A2ED092
:10C2900047D8EECF00F0EECF01F0EECF02F0EFCFB7
:10C2A00003F032D800C0EEFF01C0EEFF02C0EEFF87
:10C2B00003C0EEFF21D80050010B05E025D8020E87
:10C2C0003AD8EF8E04D020D8020E35D8EF9E14D87D
:10C2D000D8900132003218D8030E2DD800C0EFFFDD
:10C2E0001AD804E011D8030E26D8EF8EE552E5CF18
:10C2F000DAFFE7CFD9FF120013D8040E1CD8EECF17
:10C3000000F0EFCF01F01200FA0EDBCFE9FFFB0ED9
:10C31000DBCFEAFF120004D8060E0DD8EF50120052
:10C32000FC0EDBCFE9FFFD0EDBCFEAFF1200ECDFF6
:10C33000EE6AEE6A1200E926000EEA221200220ED0
:0AC340000701F16FF26B8BEF61F063
:06C34A002A0EF66E100E33
:10C35000F76E000EF86E07010900F550EA6F09004C
:10C36000F550EB6F03E1EA6701D03DD00900F550CD
:10C37000E56F0900F550E66F0900F550E76F090019
:10C380000900F550E96E0900F550EA6E0900090050
:10C390000900F550E86F0900F550E96F0900090040
:10C3A000F6CFECF7F7CFEDF7F8CFEEF7E5C7F6FFEE
:10C3B000E6C7F7FFE7C7F8FF0701E85302E1E953D3
:10C3C00007E00900F550EE6EE807F8E2E907F9D753
:10C3D000ECC7F6FFEDC7F7FFEEC7F8FF0701EA0766
:08C3E000000EEB5BBFD7120059
:08C3E800FE0EE3CFE9FFFF0E9A
:10C3F000E3CFEAFFE9CFF3FFEACFF4FFFB0EE35010
:10C4000003E1FC0EE35009E0FB0EE30602E2FC0E42
:10C41000E306FD0EE350EE6EF1D71200FE0EE3CF01
:10C42000E9FFFF0EE3CFEAFFF36AF46AEE5203E09E
:10C43000F34AF42AFBD71200FF0EE3CFF8FFE552D0
:10C44000FF0EE3CFF7FFE552FF0EE3CFF6FFE55215
:10C45000E66AE66AE66A0900F55209E0FD0EE32A9B
:10C4600005E1FE0EE32A02E1FF0EE32AF4D7FD0EFA
:10C47000E3CF39F0FE0EE3CF3AF0FF0EE3CF3BF00F
:02C480001200A8
:0EC48200D9CFE6FFDACFE6FFE1CFD9FFE2CF58
:10C49000DAFFE652E652E652E652D950FB0F006E42
:10C4A000FF0EDA20016E00C0DEFFDD6EDECFE6FF9C
:10C4B000DDCFE6FFFB0EDBCFE6FFFC0EDBCFE6FFBA
:10C4C000FD0EDBCFE6FFF3C7E6FFF4C7E6FFF8ECAF
:10C4D0004DF0006E070EE15C02E2E16AE552E16EAA
:10C4E0000050020EF3CFDBFF030EF4CFDBFF020E92
:10C4F000DBCF00F0030EDBCF01F000C0F3FF01C083
:10C50000F4FF040EE15C02E2E16AE552E16EE552FD
:0AC51000E5CFDAFFE7CFD9FF1200F4
:06C51A0012010002020004
:10C520000040D80492FD820101020001090243008B
:10C53000020100C0320904000001020201000524CA
:10C540000010010424020205240600010524010054
:10C55000010705810308000209040100020A000026
:10C5600000070502024000000705820240000004A7
:10C5700003090418035300630068006D0061006C38
:10C58000007A0048006100750073001603450069D9
:10C590000042006F00740042006F0061007200648E
:09C5A000002CC56FC573C58BC5E5
:06C5AA00D9CFE6FFDACF55
:10C5B000E6FFE1CFD9FFE2CFDAFFFB0EDBCF00F0E1
:10C5C000FC0EDBCF01F00001800E01141AE1FB0E1E
:10C5D000DBCFE9FFFC0EDBCFEAFFEECFF3FFEDCFC1
:10C5E000F4FFEE2A000EEF22F3CFE9FFF4CFEAFFCB
:10C5F000FD0EDBCFEFFFEF50016AF36E01C0F4FFD9
:10C6000010D0FB0EDB50FE0806E1FD0EDBCFE6FF8F
:10C61000E8EC63F005D0FD0EDBCFE6FF3FEC3AF02F
:0EC62000E552E552E5CFDAFFE7CFD9FF120071
:02C62E00385082
:10C630003D02F3CF34F0F4CF35F03E02F35035260F
:10C64000000EF420366E38503F02F3503626000EAE
:10C65000F420376E38504002F350372639503D02EF
:10C66000F3503526F4503622000E372239503E0260
:10C67000F3503626F450372239503F02F350372614
:10C680003A503D02F3503626F45037223A503E02DB
:0EC69000F35037263B503D02F3503726120080
:02C69E00FF0E8D
:10C6A000E124E96EFF0EE220EA6EEDCFF4FFEFCF5A
:10C6B000F3FFF46607D0600EF36404D07B0EF360E2
:10C6C00001D0F39A1200F36AF46AFF0EE124E96ED6
:10C6D000FF0EE220EA6EED6607D02F0EEF6404D065
:0AC6E0003A0EEF6001D0F32A1200B9
:06C6EA00376A366A356A6A
:10C6F000346A200EE76ED890383639363A363B36F3
:10C7000034363536363637363D50345C3E50355843
:10C710003F5036584050375809E33D50345E3E5044
:10C72000355A3F50365A4050375A382AE72EE4D708
:02C730001200F5
:0EC732004F4B0D0A000D0A004542427631338E
:10C740005F616E645F61626F766520454220466975
:10C75000726D776172652056657273696F6E2032F3
:07C760002E342E340D0A00F7
:08C76800376A366A100EE76E15
:10C77000D8903A363B36363637363F50365C4050E6
:10C78000375805E33F50365E4050375A3A2AE72E75
:04C79000F0D71200CC
:0CC79400C00EF36E00EE00F00E0E01D897
:10C7A0001200EA6002D0EE6AFCD7F350E960120092
:04C7B000EE6AFCD75A
:0CC7B4001DEE00F02DEE00F0F86A439C32
:10C7C000A5EC61F00AEC64F04AEC5FF0FBD71200D4
:10C7D000FF0EE350ADBA04D0B06AAC8EAD8A949C23
:0CC7E000ADA2FED7AE6EF36EF46A12003C
:04C7EC00F36AF46A8E
:10C7F000F32A0F0B05E0D890F336F436E804FBE19A
:02C80000120024
:0EC80200303132333435363738396162636491
:03C810006566005A
:02C81400120010
:02C81600FEFF23
:08C81800000000000000000018
:01C820000116
:0FC8210000000000000000000000000000000008
:10C8300000000000000000000000000000000000F8
:10C8400000000000000000000000000000000000E8
:10C8500000000000000000000000000000000000D8
:10C8600000000000000000000000000000000000C8
:10C8700000000000000000000000000000000000B8
:10C880000000000000920F920F920F930F930F93EE
:10C890000F930F930F930F930F930F940F940F9485
:10C8A0000F940F940F940F940F940F950F950F956D
:10C8B0000F950F950F950F890F890F890F8A0F8A92
:10C8C0000F8A0F8A0F8A0F8A0F8A0F8A0F8B0F8B9E
:10C8D0000F8B0F8B0F8B0F8B0F8B0F8B0F8C0F8C86
:10C8E0000F8C0F8C0F8C0F8C0F00010500010203C1
:10C8F00004050607000102030405060702030405F8
:02C90000060728
:00000001FF
